:020000040800F2
:1000000000C0012061B00008ADB00008ADB000082C
:10001000ADB00008ADB00008ADB0000800000000B1
:10002000000000000000000000000000ADB000086B
:10003000ADB0000800000000ADB000087D19000858
:10004000ADB00008ADB00008ADB00008ADB000081C
:10005000ADB00008ADB00008ADB00008ADB000080C
:10006000ADB00008BD190008ADB00008ADB0000883
:10007000ADB00008ADB00008ADB00008ADB00008EC
:10008000ADB00008ADB00008ADB00008ADB00008DC
:10009000ADB00008ADB00008ADB00008ADB00008CC
:1000A000ADB00008ADB00008ADB00008ADB00008BC
:1000B000ADB00008ADB00008ADB00008ADB00008AC
:1000C000ADB00008ADB00008ADB00008ADB000089C
:1000D000ADB00008ADB00008ADB00008ADB000088C
:1000E000ADB00008ADB00008ADB00008ADB000087C
:1000F000ADB00008ADB00008ADB00008ADB000086C
:10010000ADB00008ADB00008ADB00008ADB000085B
:10011000ADB00008ADB00008ADB00008ADB000084B
:10012000ADB00008ADB000089D190008AD19000879
:10013000ADB000080000000000000000ADB00008F5
:10014000ADB00008ADB00008ADB000088D190008D2
:10015000ADB00008ADB00008ADB00008ADB000080B
:10016000ADB00008ADB00008ADB00008ADB00008FB
:10017000ADB00008ADB000080000000000000000B5
:10018000ADB00008ADB0000880B483B000AF034646
:100190003960FB713B6812221A80034B18460C37FA
:1001A000BD465DF8047B70471C00002080B483B01E
:1001B00000AF03463960FB713B6804221A80034B91
:1001C00018460C37BD465DF8047B704730000020B0
:1001D00080B582B000AF03463960FB710448054921
:1001E0003A6802F035F9034B18460837BD4680BD22
:1001F00064B200087001002080B582B000AF0346F1
:100200003960FB71044805493A6802F021F9034B53
:1002100018460837BD4680BD78B20008700100203E
:1002200080B582B000AF03463960FB7104480549D0
:100230003A6802F00DF9034B18460837BD4680BDF9
:100240008CB200087001002080B582B000AF034678
:100250003960FB71044805493A6802F0F9F8034B2C
:1002600018460837BD4680BD9CB2000870010020CA
:1002700080B582B000AF03463960FB710448054980
:100280003A6802F0E5F8034B18460837BD4680BDD2
:10029000A8B200087001002080B588B000AF786077
:1002A0007B681B68B3F1A04F24D1144A134B5B6BDE
:1002B00043F080035363114A104B5B6C43F480435B
:1002C00053644FF4C053FB6002233B6100237B6106
:1002D0000023BB610A23FB6107F10C0308481946A0
:1002E00007F014F943200A2100220AF0D1FD43202F
:1002F0000AF0EAFD2037BD4680BD00BF003802404D
:100300000000024080B582B000AF78607B68D3F80F
:10031000B0237B6803F560731046194602F098F924
:100320000837BD4680BD00BF80B582B000AF7860A1
:100330000B46FB707B68D3F8B003FA7879681346F4
:10034000DB009B1A9B000B4403F5F0735B68FA78A3
:1003500011461A4602F0C6F90837BD4680BD00BFF7
:1003600080B582B000AF78600B46FB707B68D3F835
:10037000B003FA7879681346DB009B1A9B000B44A4
:1003800038339B68FA7811461A4602F007FA0837A4
:10039000BD4680BD80B582B000AF78607B68D3F881
:1003A000B033184602F0F2FA0837BD4680BD00BFF0
:1003B00080B584B000AF78600123FB737B68DB6895
:1003C000002B02D0022B03D005E00023FB7305E0D5
:1003D0000123FB7302E00123FB7300BF7B68D3F8AA
:1003E000B023FB7B1046194602F098FA7B68D3F8DD
:1003F000B033184602F062FA1037BD4680BD00BF28
:1004000080B582B000AF78607B68D3F8B03318460F
:1004100002F094FA7B681B6803F560631A467B68F8
:100420001B6803F560631B6843F001031360083722
:10043000BD4680BD80B582B000AF78607B681B6828
:1004400003F560631A467B681B6803F560631B68ED
:1004500023F0010313607B68D3F8B033184602F031
:1004600083FA0837BD4680BD80B582B000AF7860A2
:100470000B46FB707B68D3F8B023FB781046194617
:1004800002F0ACFA0837BD4680BD00BF80B582B02F
:1004900000AF78600B46FB707B68D3F8B023FB7825
:1004A0001046194602F08CFA0837BD4680BD00BFE1
:1004B00080B582B000AF78607B68D3F8B03318465F
:1004C00002F09AFA0837BD4680BD00BF80B582B001
:1004D00000AF78607B68D3F8B033184602F098FA22
:1004E0000837BD4680BD00BF80B582B000AF7860E0
:1004F0007B68D3F8B033184602F0A2FA0837BD463D
:1005000080BD00BF80B582B000AF78607B681B788B
:10051000002B3AD11F4A7B68C2F8B0337B681D4A72
:10052000C3F820221B4B4FF0A0421A60194B072240
:100530005A60184B0222DA60164B00221A61154BE2
:1005400000225A61134B02229A61124B0022DA6197
:10055000104B00221A620F4B00229A620D4B0022B0
:10056000DA620C4B00221A630A4805F0C5FF0948FD
:10057000802105F0AFFF07480021402205F05CFF15
:1005800004480121802205F057FF00231846083750
:10059000BD4680BD7003002080B582B000AF78609A
:1005A0007B68D3F82032184606F0AEF800231846D0
:1005B0000837BD4680BD00BF80B582B000AF78600F
:1005C0007B68D3F82032184606F0C0F8002318469E
:1005D0000837BD4680BD00BF80B582B000AF7860EF
:1005E000084611461A460346FB700B46BB7013467D
:1005F0003B807B68D3F82002F9783A88BB7806F014
:10060000A1FC002318460837BD4680BD80B582B0E6
:1006100000AF78600B46FB707B68D3F82022FB7834
:100620001046194606F0F6FC002318460837BD466A
:1006300080BD00BF80B582B000AF78600B46FB7014
:100640007B68D3F82022FB781046194606F0A4FEFA
:10065000002318460837BD4680BD00BF80B582B074
:1006600000AF78600B46FB707B68D3F82022FB78E4
:100670001046194606F0EAFD002318460837BD4625
:1006800080BD00BF80B582B000AF78600B46FB70C4
:100690007B68D3F82022FB781046194606F032FE1C
:1006A000002318460837BD4680BD00BF80B485B022
:1006B00000AF78600B46FB707B68D3F82032FB609C
:1006C000FB785BB2002B0BDAFB7803F07F02F96852
:1006D0001346DB009B1A9B000B4430339B790BE0E5
:1006E000FB7803F07F02F9681346DB009B1A9B003E
:1006F0000B4403F5EC739B7818461437BD465DF840
:10070000047B704780B582B000AF78600B46FB7009
:100710007B68D3F82022FB781046194606F0F0FBE0
:10072000002318460837BD4680BD00BF80B584B0A1
:1007300000AFF8607A601A460B46FB7213463B81A5
:10074000FB68D3F820123B89FA7A084611467A688A
:1007500006F020FD002318461037BD4680BD00BFBF
:1007600080B584B000AFF8607A601A460B46FB7221
:1007700013463B81FB68D3F820123B89FA7A08467E
:1007800011467A6806F090FC002318461037BD46E3
:1007900080BD00BF80B582B000AF78600B46FB70B3
:1007A0007B68D3F82022FB781046194606F0D8FC67
:1007B000034618460837BD4680BD00BF80B500AF70
:1007C00002480349002201F09DFE80BD240700205D
:1007D0000000002080B582B000AF00F04BF900F0BF
:1007E000D7F938603B68002B03D1174B03221A70EE
:1007F00026E03B6840F201129A803B6800229A7121
:100800003B680022DA71FF237B710023FB800AE042
:10081000FB883A6813447A791A727B7927337B71A3
:10082000FB880133FB80FB88B3F5007FF0D3386889
:1008300000F01AFA0346002B02D1044800F08EFBA8
:100840000837BD4680BD00BF44010020B108000844
:1008500080B500AF074B03221A70074B1B78002BA3
:1008600006D0054B1B78012B02D8044801F09AFEF4
:1008700080BD00BF44010020450100202407002066
:1008800080B500AF094B1B78032B01D101230AE08F
:10089000064B1B78022B05D0642001F01DF8FFF7F2
:1008A000D7FFFEE70023184680BD00BF44010020AB
:1008B00080B584B000AF78601F4B1B78022B00D945
:1008C00037E01D4B1B78002B02D17B68002B05D134
:1008D000642001F001F8FFF7BBFFFEE77B689B880F
:1008E00040F20112934205D0642000F0F5FFFFF7BB
:1008F000AFFFFEE7FF237B730023FB8112E0FB8940
:100900007A6813441B7A7A7B9A4205D0642000F0FF
:10091000E3FFFFF79DFFFEE77B7B27337B73FB89BC
:100920000133FB81FB89B3F5007FE8D3786800F0E1
:1009300005F81037BD4680BD4401002080B582B067
:1009400000AF78600B4B01221A707B6801229A80FD
:100950007B6800229A717B680122DA71786800F066
:1009600083F90346002B02D1034800F0F7FA083759
:10097000BD4680BD440100207D09000880B584B0DB
:1009800000AF78600023FB73274B1B78022B00D944
:1009900047E0254B1B78012B02D17B68002B05D14A
:1009A000642000F099FFFFF753FFFEE77B689B8808
:1009B000022B05D0642000F08FFFFFF749FFFEE710
:1009C0007B681B7A012B04D10123FB73174BBB609F
:1009D00000BF786800F012F9FB7B002B05D1642082
:1009E00000F07AFFFFF734FFFEE7114B1B78002B76
:1009F0000AD00F4B1B78FA7B9A4205D0642000F096
:100A00006BFFFFF725FFFEE7074B02221A70084A2B
:100A1000FB7B13700748B96801F09EFD054801F0A3
:100A2000B5FD1037BD4680BD4401002034000020D4
:100A3000450100202407002080B500AF0A4B1B7839
:100A4000002B03D0084B1B78012B05D9642000F044
:100A500043FFFFF7FDFEFEE7044801F0A3FD044855
:100A600000F056F880BD00BF45010020240700209B
:100A70003D09000880B500AF1F4B00221A701F4BC4
:100A800000221A701E4B1F4A1A601D4B002283F869
:100A900051201B4B4FF482725A60194B00229A600E
:100AA000174B4FF40062DA60154B00221A61144BA9
:100AB00000225A61124B4FF400729A61104B2022AF
:100AC000DA610F4B00221A620D4B00225A620C4B66
:100AD0004FF400529A620A4B0722DA62084804F087
:100AE00051FD094B1B6903F00803002B02D1074B92
:100AF00001221A7080BD00BF5C0B0020500900204D
:100B0000680D002000300140000002405801002024
:100B100080B582B000AF7860194B1B78082B01D9E3
:100B2000012328E0174B1B68002B08D0642000F03D
:100B3000D3FE134B09221A70FFF78AFEFEE7124B11
:100B40001B78002B07D1104B01221A707B680E48CE
:100B5000984700230FE00D4B1B78002B07D10B4B60
:100B600001221A707B6809489847002303E0054A70
:100B70007B681360002318460837BD4680BD00BF60
:100B80004C010020500100205C0B00205009002087
:100B900080B582B000AF154B1B78082B01D900231C
:100BA00020E0134B1B68002B01D00023FB71114B7D
:100BB0001B78002B04D10F4B01221A700D4B11E052
:100BC0000D4B1B78002B04D10B4B01221A700A4BE2
:100BD00008E0642000F080FE044B09221A70FFF741
:100BE00037FEFEE718460837BD4680BD4C010020A1
:100BF000480100205C0B00205009002080B584B023
:100C000000AF7860144B1B78082B00D921E07B687B
:100C1000124A93420CD07B68114A934208D0642058
:100C200000F05AFE0C4B09221A70FFF711FEFEE786
:100C30000C4B1B68002B09D00A4B1B68FB60094B4F
:100C400000221A60FB687868984702E07B680022FF
:100C50001A701037BD4680BD4C0100205C0B00208F
:100C6000500900205001002080B582B000AF7860AC
:100C7000374B1B78082B01D9012364E07B68354A88
:100C800093420CD07B68344A934208D0642000F031
:100C900023FE2F4B09221A70FFF7DAFDFEE77B686F
:100CA0001B78012B08D17B689B88002B04D07B68C4
:100CB0009B88B3F5817F08D3642000F00DFE244BA0
:100CC00009221A70FFF7C4FDFEE7244B1B68002BB6
:100CD00008D0642000F000FE1D4B09221A70FFF7B7
:100CE000B7FDFEE71A4B1B78002B07D0002B20DB4B
:100CF000042B1EDC194A7B68136023E0144B01228D
:100D00001A70174A7B681360154B1B689A79154B4C
:100D10001A70134B1B68DA79134B1A70134B1B783C
:100D2000002B05D0114B00221A7000F0ADF909E03C
:100D300008E0642000F0D0FD054B09221A70FFF78F
:100D400087FDFEE7002318460837BD4680BD00BF7B
:100D50004C0100205C0B00205009002048010020BD
:100D6000580B0020640D00204C0900205801002081
:100D700080B584B000AF78606F4B10229A616F4BE2
:100D80001B78082B00D9D3E06C4B1B78022B0DD1BC
:100D90006A4B03221A706A4B1B78002B05D0684BF4
:100DA00000221A7000F09AF9C2E0C1E0634B1B7890
:100DB000042B3ED1634B1B68002B0CD0624B1B688D
:100DC000002B08D1642000F087FD5C4B09221A70CB
:100DD000FFF73EFDFEE75D4B1B681846FFF70EFF71
:100DE000564B1B78092B00D1A2E0574B1B68002BF8
:100DF00014D0524B01221A70534B1B68534A136094
:100E0000514B00221A604E4B1B78002B05D04C4BE7
:100E100000221A7000F038F98AE089E0474B00227E
:100E20001A704B4B1B68002B02D000F0BDF87FE01E
:100E30007EE0424B1B78062B21D1444B1B689B88DC
:100E4000002B05D0414B1B689B88B3F5817F08D3ED
:100E5000642000F041FD394B09221A70FFF7F8FCBD
:100E6000FEE7364B07221A70354B1B78002B05D056
:100E7000334B00221A7000F0B1F959E058E02F4BC3
:100E80001B78082B4BD12D4B00221A70304B1B685E
:100E9000002B08D1642000F01FFD284B09221A7096
:100EA000FFF7D6FCFEE7294B1B689B79022B0FD17D
:100EB000264B1B68DB79012B0AD1244B1B68184693
:100EC000FFF79CFE224B00221A60FFF7B5FD2FE0D2
:100ED0001E4B1B689B791A461E4B1B78534003F030
:100EE0007F03002B06D1194B1B68DA791A4B1B784C
:100EF0009A4208D0642000F0EFFC104B09221A70CF
:100F0000FFF7A6FCFEE7124B1B68FB60104B0022AC
:100F10001A600E4B1A68FB681046984708E0642078
:100F200000F0DAFC054B09221A70FFF791FCFEE78E
:100F30001037BD4680BD00BF000002404C010020BC
:100F4000580100205001002048010020580B0020CB
:100F500054010020640D00204C09002080B582B0AF
:100F600000AF78600E4B1B78082B01D9012312E0EB
:100F70000C4B1B68002B08D0642000F0ADFC084B24
:100F800009221A70FFF764FCFEE7064A7B681360CB
:100F900000F00AF8034618460837BD4680BD00BF7A
:100FA0004C0100205401002080B500AF134B1B788A
:100FB000082B01D901231EE0104B1B78042B08D904
:100FC000642000F089FC0D4B09221A70FFF740FCE9
:100FD000FEE70A4B1B78002B0CD1084B05221A7038
:100FE000074B1B78002B05D0054B00221A700548D3
:100FF000FFF78EFD0023184680BD00BF4C01002086
:10100000580100204911000880B500AF1B4B1B7828
:10101000082B00D930E0194B1B78072B23D801A2ED
:1010200052F823F0451000084D1000086710000822
:1010300053100008671000085910000867100008D6
:10104000611000080E4B01221A7015E000F01CF828
:1010500012E000F043F80FE00A48FFF759FD0BE0FB
:1010600000F0BCF808E0642000F036FC034B0922D5
:101070001A70FFF7EDFBFEE780BD00BF4C010020BA
:10108000580100204911000880B500AF0E4B022224
:101090001A700E4B4FF480129A610D4B1B6804338B
:1010A0000C4819460C4A022304F0D2FA0346002BDE
:1010B00008D0642000F010FC034B09221A70FFF7DF
:1010C000C7FBFEE780BD00BF4C01002000000240CE
:1010D000580B0020680D00204809002080B500AFA3
:1010E000154B04221A70154B4FF480129A61144B61
:1010F0001B689B88C82B02D90F4B04221A70104B17
:101100001B68991D0E4B1B689A1D0D4B1B689B8815
:10111000022B38BF02239BB20A4804F099FA034617
:10112000002B08D0642000F0D7FB034B09221A7073
:10113000FFF78EFBFEE780BD4C010020000002405F
:10114000580B0020680D002080B582B000AF786099
:101150001D4B1B78082B00D932E01B4B1B78052B4D
:1011600008D0642000F0B8FB174B09221A70FFF773
:101170006FFBFEE7144B06221A70144A7B6813605B
:10118000124B1B6800229A80114B4FF480129A6117
:10119000104B00221A600D4B1B6804330E480D499A
:1011A0001A46022304F054FA0346002B08D06420A8
:1011B00000F092FB044B09221A70FFF749FBFEE78F
:1011C0000837BD4680BD00BF4C010020580B0020F1
:1011D0000000024048090020680D002080B500AFE3
:1011E000114B08221A70114B4FF480129A61104B68
:1011F0001B68991D0E4B1B689A1D0D4B1B689B8825
:10120000022B38BF02239BB20A4804F021FA03469E
:10121000002B08D0642000F05FFB034B09221A70FA
:10122000FFF716FBFEE780BD4C01002000000240E6
:10123000580B0020680D002080B582B000AF7860A8
:10124000094B10229A61094B1B78082B00D908E042
:10125000642000F041FB054B09221A70FFF7F8FAF1
:10126000FEE70837BD4680BD000002404C0100206B
:1012700080B582B000AF7860084B1B78082B00D98E
:1012800008E0642000F028FB044B09221A70FFF7E5
:10129000DFFAFEE70837BD4680BD00BF4C010020E5
:1012A00080B584B000AF7860FFF7EAFA0346002B00
:1012B00001D001231FE0124A7B681360FFF768FC2E
:1012C000F860FB68002B01D1012314E0FB680122C8
:1012D0009A80FB6801229A71FB680022DA71F86833
:1012E000FFF7C2FC0346002B04D10648FFF736FE89
:1012F000034600E0012318461037BD4680BD00BFFD
:10130000CC0D00200913000880B582B000AF7860D2
:10131000FFF7B6FA0346002B00D01EE07B68002BD7
:1013200004D10F4B1B680120984716E07B689B880F
:10133000022B03D17B681B7A002B07D07868FFF75C
:101340005DFC074B1B680120984706E07868FFF7B3
:1013500055FC034B1B68002098470837BD4680BDED
:10136000CC0D002080B584B000AF7860FFF788FA1C
:101370000346002B01D001231FE0124A7B68136053
:10138000FFF706FCF860FB68002B01D1012314E095
:10139000FB6801229A80FB6801229A71FB68012296
:1013A000DA71F868FFF760FC0346002B04D10648A9
:1013B000FFF7D4FD034600E0012318461037BD4671
:1013C00080BD00BFC80D0020CD13000880B584B0DB
:1013D00000AF7860FFF754FA0346002B00D022E0FC
:1013E0007B68002B06D1114B1B68002000210022D6
:1013F000984718E07B689B88052B06D00B4B1B6831
:1014000000200021002298470DE07B6808331B680C
:10141000FB607B680C331B68BB60044B1B687868FF
:10142000F968BA6898471037BD4680BDC80D0020DE
:1014300080B586B000AFF860C7E90023FFF720FA57
:101440000346002B01D0012333E01C4B00221A601D
:101450001B4B00221A701B4A7B6A13601A4AFB68F6
:101460001360FFF795FB78617B69002B01D10123A5
:101470001FE07B6907229A807B6901229A717B6950
:101480000222DA717B6903F10801D7E90023C1E97F
:1014900000237B6910333A6A1A607869FFF7E4FB2E
:1014A0000346002B04D10948FFF758FD034600E02E
:1014B000012318461837BD4680BD00BFC00D00206F
:1014C000C40D0020D40D0020CC0D0020091300080D
:1014D00080B582B000AF7860FFF7D2F90346002BE9
:1014E00001D0012321E0134A7B681360124B1B7863
:1014F000002B01D0002318E00F4B01221A700F4B74
:101500001B68002B0DD00B4B1B68002B09D00B4B1D
:101510001B68184600F016F8084B00221A600023DA
:1015200003E00748FFF71AFD034618460837BD4693
:1015300080BD00BFD00D0020C40D0020C00D0020D4
:101540004515000880B584B000AF7860254B0022B7
:101550001A70FFF795F90346002B00D03EE0224BAE
:101560001B68002B03D1214A7B68136036E07B683F
:10157000002B05D11C4B1B680020002198472DE053
:101580007B689B88013B9BB25B00FB817B689B79FE
:10159000DBB25BB2002B08DA7B689B88012B04D995
:1015A000FA89134B1B689A4205D90F4B1B68002020
:1015B0000021984712E00E4B1A68FB89D31A0C4A97
:1015C0001360094B1B68FA89786811469847084BE5
:1015D0001B68002B02D00020FFF77AFF1037BD46B2
:1015E00080BD00BFC40D0020D00D0020C00D002024
:1015F000D40D002080B586B000AFF860C7E90023A5
:10160000FFF73EF90346002B01D001232AE0174AD9
:10161000FB681360FFF7BCFA78617B69002B01D18E
:1016200001231FE07B6907229A807B6901229A715E
:101630007B690322DA717B6903F10801D7E9002392
:10164000C1E900237B6910333A6A1A607869FFF7B1
:101650000BFB0346002B04D10548FFF77FFC034634
:1016600000E0012318461837BD4680BDCC0D002090
:101670007516000880B584B000AF7860FFF700F9F8
:101680000346002B00D026E07B68002B04D1134BCF
:101690001B68012098471EE07B689B88022B07D1BE
:1016A0007B681B7A002B0BD07B681B7A022B07D040
:1016B0007868FFF7A3FA094B1B68012098470AE0F6
:1016C0007B681B7AFB737868FFF798FA034B1B68FB
:1016D000FA7B104698471037BD4680BDCC0D0020E0
:1016E00080B582B000AF78603960FFF7C9F8034673
:1016F000002B01D0012317E03B6803F00103002B0E
:1017000001D0012310E03B685B089BB201339AB221
:101710007B689A807B6881229A717B680322DA71E8
:101720007868FFF7A1FA034618460837BD4680BD22
:1017300080B500AF00F00CF809F0FCFB00F054F8A5
:1017400000F0B8F8FFF73AF8FFF744F8FEE700BFFB
:1017500080B592B000AF224A214B1B6C43F08053FE
:101760001364204A1F4B1B6823F4404343F4004397
:1017700013600123BB610123FB6102233B634FF430
:1017800080037B630823BB634FF4A873FB630423CC
:101790003B6407237B6407F11803184604F058FAEA
:1017A0000346002B00D0FEE70D237B600223BB60C5
:1017B0000023FB604FF4A0533B614FF480537B61E7
:1017C0003B1D1846022104F027FC0346002B00D0E5
:1017D000FEE7042009F092FB4837BD4680BD00BFFC
:1017E000003802400070004080B586B000AF2C4A3F
:1017F0002B4B1B6B43F001031363294A284B1B6BD4
:1018000043F002031363264A254B1B6B43F004038A
:101810001363234A224B1B6B43F00803136341F607
:10182000FF737B600023BB600123FB6000233B61EF
:1018300000237B613B1D1B48194605F067FE4FF6F0
:10184000E7737B603B1D1848194605F05FFE4FF6B5
:10185000FF737B603B1D1548194605F057FE3B1D85
:101860001348194605F052FE10237B600323BB602A
:101870003B1D0E48194605F049FE4FF480537B602E
:101880000123BB600023FB603B1D0848194605F09F
:101890003DFE064B4FF480529A611837BD4680BD1D
:1018A00000380240000002400004024000080240EC
:1018B000000C024080B500AF064B4FF080529A6199
:1018C0004FF4FA7009F088FB024B4FF480529A6192
:1018D00080BD00BF0008024080B483B000AF034663
:1018E000FB80094AFB881380FB88002B06D1074B3D
:1018F00000221A70064B4FF480529A610C37BD4695
:101900005DF8047B704700BF5A0100205E01002093
:101910000008024080B400AF144B1B88002B21D07C
:10192000134B1B8801339AB2114B1A80104B1A8843
:101930000E4B1B889A4215D30D4B00221A800D4B7B
:101940001B78002B07D00B4B00221A700A4B4FF468
:1019500080529A6106E0074B01221A70064B4FF045
:1019600080529A61BD465DF8047B70475A010020A1
:101970005C0100205E0100200008024080B500AF3D
:1019800009F010FBFFF7C6FF80BD00BF80B500AFB8
:10199000014804F003FF80BD7003002080B500AF54
:1019A000014806F013F880BDD80D002080B500AFC7
:1019B000014806F00BF880BD280E002080B500AF6E
:1019C000024B08225A61FFF71FFB80BD003C01401B
:1019D00080B500AF4FF0FF300221002209F058FA25
:1019E00080BD00BF80B588B000AF78607B681B68A1
:1019F000564A934240F0A780554A554B5B6C43F4DE
:101A000080535364524A524B1B6B43F4800313635D
:101A1000E023FB6002233B6102237B610123BB6166
:101A20000523FB6107F10C034A48194605F06EFDDA
:101A3000484B10229A611023FB6001233B61002375
:101A40007B6107F10C034348194605F05FFD08234D
:101A5000FB60414B3B6101237B6107F10C033D4877
:101A6000194605F053FD09200A21002209F010FA59
:101A7000092009F029FA7B68384A1A64374B384A3A
:101A80001A60364A7B689363344B4FF0C0625A60E9
:101A9000324B40229A60314B0022DA602F4B4FF4D8
:101AA00080621A612D4B4FF400625A612B4B4FF448
:101AB00000529A61294B0022DA61284B4FF48032A0
:101AC0001A62264B00225A62244805F0B5FE3B20DC
:101AD0000A21002209F0DCF93B2009F0F5F97B68C6
:101AE000204A5A641F4B204A1A601E4A7B6893633F
:101AF0001C4B4FF0C0625A601A4B00229A60194B7F
:101B00000022DA60174B4FF480621A61154B4FF4D4
:101B100000625A61134B4FF400529A61114B00223C
:101B2000DA61104B4FF480321A620E4B00225A6277
:101B30000C4805F081FE3A200A21002209F0A8F99C
:101B40003A2009F0C1F92037BD4680BD0030014080
:101B5000003802400000024000002110280E002042
:101B600058640240D80D00204064024080B584B023
:101B700000AFF860B9601346FB80FB680222C3F82F
:101B8000F421FA88FB689A61FA88FB68DA61FB88BD
:101B9000F8680021BA68FEF7C9FD0023184610371F
:101BA000BD4680BD80B584B000AFF860B960134613
:101BB000FB80FB88F8680021BA68FEF7B7FD0023B8
:101BC00018461037BD4680BD80B584B000AFF860C0
:101BD000B9601346FB80FB88F8680021BA68FEF7FD
:101BE000BFFD002318461037BD4680BD80B582B0CA
:101BF00000AF78607B680422C3F8F4217868002184
:101C000000220023FEF792FD002318460837BD4648
:101C100080BD00BF80B582B000AF78607B680522D0
:101C2000C3F8F4217868002100220023FEF798FD14
:101C3000002318460837BD4680BD00BF80B584B07C
:101C400000AF786039600023FB733B685B78092B39
:101C500039D801A252F823F0A91C0008BD1C0008C5
:101C6000C71C0008B31C0008C71C00088B1C000818
:101C7000811C0008C71C00089F1C0008951C000858
:101C80007868396800F036F922E07868396800F041
:101C90002DFA1DE07868396800F066FA18E0786877
:101CA000396800F0EBFA13E07868396800F018FB47
:101CB0000EE07868396800F03DFB09E07868396823
:101CC00000F052FB04E07868396800F0B1FB00BF17
:101CD000FB7B18461037BD4680BD00BF80B584B081
:101CE00000AF786039600023FB737B6893F8FC31A8
:101CF000032B1CD13B689B88DBB2012B11D87B687E
:101D0000D3F814329B687868396898473B68DB8859
:101D1000002B0BD1FB7B002B08D17868FFF766FF07
:101D20000AE07868396800F083FB05E004E0786831
:101D3000396800F07DFB00BF002318461037BD4610
:101D400080BD00BF80B584B000AF786039600023EB
:101D5000FB733B689B88BB733B681B7803F0600395
:101D6000202B08D17B68D3F814329B6878683968D7
:101D700098470023B9E03B685B78012B39D0032BEF
:101D800002D0002B6AD0AFE07B6893F8FC31022BC5
:101D900002D0032B0DD026E0BB7B002B08D0BB7BF1
:101DA000802B05D0BB7B78681946FEF757FC1FE0F7
:101DB0001EE03B685B88002B0AD1BB7B002B07D061
:101DC000BB7B802B04D0BB7B78681946FEF746FCB2
:101DD0007B68D3F814329B687868396898477868CC
:101DE000FFF704FF04E07868396800F021FB00BFCA
:101DF0007AE07B6893F8FC31022B02D0032B0DD0E4
:101E000026E0BB7B002B08D0BB7B802B05D0BB7BA7
:101E100078681946FEF722FC1FE01EE03B685B88ED
:101E2000002B14D1BB7B03F07F03002B0BD0BB7BBB
:101E300078681946FEF726FC7B68D3F814329B6855
:101E40007868396898477868FFF7D0FE05E004E0C5
:101E50007868396800F0ECFA00BF45E07B6893F8D9
:101E6000FC31022B02D0032B0CD037E0BB7B03F0FC
:101E70007F03002B05D0BB7B78681946FEF7EEFB8D
:101E800031E030E0BB7B5BB2002B08DABB7B03F0B8
:101E90007F0301331B017A681344043307E0BB7BE3
:101EA00003F07F0310331B017A6813440433BB60D3
:101EB000BB7B78681946FEF7F9FB0346002B03D07D
:101EC000BB6801221A6002E0BB6800221A60BB688E
:101ED000786819460222FFF749FE04E078683968FD
:101EE00000F0A6FA00BF00BFFB7B18461037BD46C6
:101EF00080BD00BF80B584B000AF786039603B68BA
:101F00005B881B0A9BB2013B062B00F2D18001A229
:101F100052F823F0311F00084B1F00088B1F0008E8
:101F2000B1200008B12000085D20000883200008CF
:101F30007B68D3F810321B687A68117C07F10A02BB
:101F4000084611469847F860B7E07B681B7C002B79
:101F50000DD17B68D3F81432DB6A07F10A02104610
:101F60009847F860FB68013302221A70A5E07B688D
:101F7000D3F814321B6B07F10A0210469847F86039
:101F8000FB68013302221A7097E03B685B88DBB282
:101F9000052B5DD801A252F823F000BFB51F000841
:101FA000CF1F0008E91F0008032000081D200008BB
:101FB000372000087B68D3F810325B687A68117CA0
:101FC00007F10A02084611469847F86045E07B6829
:101FD000D3F810329B687A68117C07F10A02084630
:101FE00011469847F86038E07B68D3F81032DB6818
:101FF0007A68117C07F10A02084611469847F86092
:102000002BE07B68D3F810321B697A68117C07F1EA
:102010000A02084611469847F8601EE07B68D3F82C
:1020200010325B697A68117C07F10A020846114692
:102030009847F86011E07B68D3F810329B697A68A2
:10204000117C07F10A02084611469847F86004E03F
:102050007868396800F0ECF944E02EE07B681B7C7E
:10206000002B09D17B68D3F814329B6B07F10A026D
:1020700010469847F86020E07868396800F0D8F991
:1020800030E07B681B7C002B0DD17B68D3F81432C9
:102090005B6B07F10A0210469847F860FB68013352
:1020A00007221A7009E07868396800F0C1F919E070
:1020B0007868396800F0BCF914E07B89002B11D0F6
:1020C0003B68DB88002B0DD03B68DA887B89934224
:1020D00028BF13469BB27B817B897868F9681A46D2
:1020E000FFF744FD1037BD4680BD00BF80B584B00A
:1020F00000AF786039603B689B88002B2DD13B682E
:10210000DB88002B29D13B685B88DBB203F07F03BF
:10211000FB737B6893F8FC31032B04D17868396832
:1021200000F086F918E07B68FA7B83F8FE21FB7BE0
:1021300078681946FEF7E6FA7868FFF757FDFB7BEB
:10214000002B04D07B68022283F8FC2104E07B682A
:10215000012283F8FC2104E003E07868396800F08C
:1021600067F91037BD4680BD80B582B000AF78609A
:1021700039603B685B88DAB23F4B1A703E4B1B7884
:10218000012B04D97868396800F052F970E07B6857
:1021900093F8FC31022B02D0032B23D063E0364BA3
:1021A0001B78002B1AD0344B1B781A467B685A6078
:1021B0007B68032283F8FC212F4B1B787868194633
:1021C00000F012FA0346022B04D17868396800F057
:1021D0002FF94DE07868FFF709FD49E07868FFF7CF
:1021E00005FD45E0244B1B78002B12D17B680222B1
:1021F00083F8FC21204B1B781A467B685A601E4BE3
:102200001B787868194600F00FFA7868FFF7EEFC43
:1022100028E0194B1B781A467B685B689A421DD0F0
:102220007B685B68DBB27868194600F0FDF9124BF9
:102230001B781A467B685A600F4B1B7878681946E2
:1022400000F0D2F90346022B04D17868396800F017
:10225000EFF80DE07868FFF7C9FC03E07868FFF756
:10226000C5FC05E004E07868396800F0E1F800BFDB
:102270000837BD4680BD00BF5F01002080B582B039
:1022800000AF786039603B68DB88012B04D0786848
:10229000396800F0CDF81FE07B6893F8FC31022B21
:1022A00002D0032B0BD012E07B6800229A607B687F
:1022B0000833786819460122FFF758FC0CE07B6868
:1022C0000433786819460122FFF750FC04E078686F
:1022D000396800F0ADF800BF0837BD4680BD00BFCB
:1022E00080B582B000AF786039607B6893F8FC31CC
:1022F000023B012B15D87B680122DA607B68D3F89A
:102300000432002B05D07B68DB6843F002027B6857
:10231000DA607B680C33786819460222FFF726FCE6
:1023200004E07868396800F083F800BF0837BD46DC
:1023300080BD00BF80B582B000AF786039603B6877
:102340005B88012B0DD17B680122C3F804227B68D6
:10235000D3F814329B687868396898477868FFF733
:1023600045FC0837BD4680BD80B582B000AF7860BF
:1023700039607B6893F8FC31023B012B13D83B6832
:102380005B88012B0ED17B680022C3F804227B6896
:10239000D3F814329B687868396898477868FFF7F3
:1023A00025FC05E004E07868396800F041F800BFDA
:1023B0000837BD4680BD00BF80B483B000AF7860F1
:1023C00039603B681A787B681A703B685A787B687A
:1023D0005A703B6802331B789AB23B6803331B7810
:1023E0009BB21B029BB213449AB27B685A803B6833
:1023F00004331B789AB23B6805331B789BB21B02EF
:102400009BB213449AB27B689A803B6806331B7870
:102410009AB23B6807331B789BB21B029BB21344F2
:102420009AB27B68DA800C37BD465DF8047B704752
:1024300080B582B000AF7860396078688021FEF79F
:102440000DF978680021FEF709F90837BD4680BD0F
:1024500080B586B000AFF860B9607A600023FB7584
:10246000FB68002B33D0F86800F034F803460133E2
:102470009BB25B009AB27B681A80FB7D5A1CFA758E
:102480001A46BB6813447A681288D2B21A70FB7D70
:102490005A1CFA751A46BB68134403221A7012E0DC
:1024A000FB7D5A1CFA751A46BB681A44FB68591C16
:1024B000F9601B781370FB7D5A1CFA751A46BB68CD
:1024C000134400221A70FB681B78002BE8D11837E0
:1024D000BD4680BD80B485B000AF78600023FB733B
:1024E00005E0FB7B0133FB737B6801337B607B681A
:1024F0001B78002BF5D1FB7B18461437BD465DF8E1
:10250000047B704780B584B000AFF860B9601346B3
:10251000FB71FB68002B01D1022319E0FB6800224C
:10252000C3F81422FB680022C3F81822BB68002BF2
:1025300003D0FB68BA68C3F81022FB68012283F855
:10254000FC21FB68FA791A70F868FDF7DBFF0023BD
:1025500018461037BD4680BD80B485B000AF7860A6
:1025600039600023FB733B68002B06D07B683A6818
:10257000C3F814220023FB7301E00223FB73FB7BEF
:1025800018461437BD465DF8047B704780B582B0AD
:1025900000AF78607868FDF7FFFF00231846083722
:1025A000BD4680BD80B582B000AF78607B68D3F84F
:1025B00014325B687A685268D2B2786811469847DC
:1025C0007868FDF7F9FF002318460837BD4680BD3F
:1025D00080B483B000AF7860002318460C37BD4646
:1025E0005DF8047B704700BF80B584B000AF7860B1
:1025F0000B46FB700223FB737B68D3F81432002B6D
:102600000CD07B68D3F814321B68FA7878681146CE
:1026100098470346002B01D10023FB73FB7B184630
:102620001037BD4680BD00BF80B582B000AF786076
:102630000B46FB707B68D3F814325B68FA787868D5
:1026400011469847002318460837BD4680BD00BF95
:1026500080B582B000AF786039607B6803F50273A3
:1026600018463968FFF7A8FE7B680122C3F8F421F9
:102670007B68B3F80E321A467B68C3F8F8217B6892
:1026800093F8083203F01F03012B0BD0022B11D05B
:10269000002B17D17B6803F5027378681946FFF7A2
:1026A000CDFA1AE07B6803F5027378681946FFF7E4
:1026B00015FB12E07B6803F5027378681946FFF793
:1026C00041FB0AE07B6893F8083223F07F03DBB21A
:1026D00078681946FDF7C2FF00BF00231846083787
:1026E000BD4680BD80B586B000AFF8600B467A600D
:1026F000FB72FB7A002B38D1FB6803F582737B6198
:10270000FB68D3F8F431032B42D17B699A687B696B
:10271000DB689A4214D97B699A687B69DB68D21AB4
:102720007B699A607B69DA687B699B68934228BF02
:1027300013469BB2F86879681A46FFF745FA27E016
:10274000FB68D3F814321B69002B0AD0FB6893F89E
:10275000FC31032B05D1FB68D3F814321B69F868F0
:102760009847F868FFF742FA12E0FB68D3F8143292
:102770009B69002B0CD0FB6893F8FC31032B07D12D
:10278000FB68D3F814329B69FA7AF86811469847C7
:10279000002318461837BD4680BD00BF80B586B0FF
:1027A00000AFF8600B467A60FB72FB7A002B6CD1AD
:1027B000FB6814337B61FB68D3F8F431022B57D1EB
:1027C0007B699A687B69DB689A420FD97B699A6852
:1027D0007B69DB68D21A7B699A607B699B689BB2D4
:1027E000F86879681A46FFF7DDF905E0F868002116
:1027F00000220023FDF7B4FF7B695B687A69D26829
:10280000B3FBF2F102FB01F29B1A002B16D17B699C
:102810005A687B69DB689A4210D37B695A68FB6807
:10282000D3F8F8319A4209D2F86800210022FFF764
:10283000B9F9FB680022C3F8F82105E0F868002127
:1028400000220023FDF78CFFFB68D3F81432DB680D
:10285000002B0AD0FB6893F8FC31032B05D1FB68F1
:10286000D3F81432DB68F8689847F868FFF7D2F9B4
:10287000FB6893F80032012B1AD1F868FFF7A8FE25
:10288000FB68002283F8002212E0FB68D3F81432C0
:102890005B69002B0CD0FB6893F8FC31032B07D14C
:1028A000FB68D3F814325B69FA7AF86811469847E6
:1028B000002318461837BD4680BD00BF80B582B0E2
:1028C00000AF78607868002100224023FDF784FE85
:1028D0007B684022C3F810217868802100224023C1
:1028E000FDF77AFE7B6840221A627B68012283F83A
:1028F000FC217B68D3F81832002B09D07B68D3F811
:1029000014325B687A685268D2B278681146984788
:10291000002318460837BD4680BD00BF80B483B091
:1029200000AF78600B46FB707B68FA781A7400235E
:1029300018460C37BD465DF8047B704780B483B001
:1029400000AF78607B6893F8FC217B6883F8FD21F9
:102950007B68042283F8FC21002318460C37BD460F
:102960005DF8047B704700BF80B483B000AF78602F
:102970007B6893F8FD217B6883F8FC2100231846CF
:102980000C37BD465DF8047B704700BF80B582B050
:1029900000AF78607B6893F8FC31032B0BD17B6828
:1029A000D3F81432DB69002B05D07B68D3F81432DE
:1029B000DB6978689847002318460837BD4680BD14
:1029C00080B483B000AF78600B46FB7000231846DC
:1029D0000C37BD465DF8047B704700BF80B483B000
:1029E00000AF78600B46FB70002318460C37BD46DD
:1029F0005DF8047B704700BF80B483B000AF78609F
:102A0000002318460C37BD465DF8047B704700BFB5
:102A100080B582B000AF78607B68012283F8FC212A
:102A20007B68D3F814325B687A685268D2B27868EF
:102A300011469847002318460837BD4680BD00BFA1
:102A400080B582B000AF78607B68D3F814329B6A9F
:102A500078689847002318460837BD4680BD00BFF8
:102A600080B584B000AFF8607A603B600B46FB72C3
:102A7000814AFB681360814A7B681360804AFB7A55
:102A80001370804A3B681360FB68D3F818327E4AA3
:102A900013607B681B785A2B00F2DE8001A252F88B
:102AA00023F000BF112C0008592C0008592C0008F5
:102AB000172C0008592C0008592C0008592C000824
:102AC000592C0008592C0008592C0008592C0008D2
:102AD000592C0008592C0008592C0008592C0008C2
:102AE000592C0008592C0008592C00081D2C0008EE
:102AF000592C0008592C0008592C0008592C0008A2
:102B0000592C0008592C0008592C00082F2C0008BB
:102B1000232C0008592C0008592C0008292C0008E7
:102B2000592C0008592C0008592C0008592C000871
:102B30003B2C0008592C0008412C0008592C000897
:102B4000592C0008472C0008592C00084D2C00086F
:102B5000592C0008592C0008592C0008592C000841
:102B6000532C0008592C0008592C0008592C000837
:102B7000592C0008592C0008592C0008592C000821
:102B8000592C0008592C0008592C0008592C000811
:102B9000592C0008592C0008592C0008592C000801
:102BA000592C0008592C0008592C0008592C0008F1
:102BB000592C0008592C0008592C0008592C0008E1
:102BC000592C0008592C0008592C0008592C0008D1
:102BD000592C0008592C0008592C0008592C0008C1
:102BE000592C0008592C0008592C0008592C0008B1
:102BF000592C0008592C0008592C0008592C0008A1
:102C0000592C0008592C0008592C0008352C0008B4
:102C100000F03CF82CE000F09DFA29E000F09AF872
:102C200026E000F06DFB23E000F06AFB20E000F0FE
:102C30002DFA1DE000F05CFA1AE000F089F917E0C7
:102C400000F0E0F814E000F06BFB11E000F0B2FCE3
:102C50000EE000F035FE0BE0FB7AF868194605221D
:102C6000202300F00FFB074B1B684FF0FF30984705
:102C70001037BD4680BD00BF880E00207C0E0020AE
:102C8000800E0020840E0020780E002080B500AF5A
:102C9000134B1B68DB69002B0FD0124B1A68124BC9
:102CA0001B78104619460522202300F0EBFA0F4B43
:102CB0001B684FF0FF30984710E00B4B1B78002B40
:102CC00003D0012000F016F808E00948FEF7E8FA02
:102CD0000346002B02D0012000F00CF880BD00BF9D
:102CE000780E0020880E0020800E0020840E002028
:102CF000F52C000880B582B000AF0346FB71FB796C
:102D0000002B13D00F4B1A680F4B1B781046194637
:102D100002223A2300F0B6FA0C4B1B6805221A7205
:102D20000B4B1B684FF0FF30984707E0074B1B68C1
:102D300000225A81064B1B68002098470837BD4681
:102D400080BD00BF880E0020800E0020780E00207D
:102D5000840E002080B584B000AFFDF719FF7860C5
:102D6000234B1B687A681A61214B1B687A6808320A
:102D7000DA60204B1B6801331B7803F00103002B42
:102D800004D01D4BFB6007237B8114E01B4BFB60D1
:102D9000FB6804331B789BB205337B81154B1B68A2
:102DA00004331B789BB27A899A4204D3114B1B6877
:102DB00004331B787B810E4B1B687A895A810CE0A7
:102DC0007B89013B7B810A4B1B68DA687B89134452
:102DD0007A89F9680A4412781A707B89002BEFD13E
:102DE000074B1B68002098471037BD4680BD00BFC9
:102DF000780E00207C0E0020B8B2000840B2000817
:102E0000840E002080B500AF0548FEF7ABFA0346FC
:102E1000002B04D000200021002200F003F880BD28
:102E2000252E000880B584B000AFF860B9607A60E4
:102E3000FB68002B0FD1424B1A68424B1B7810469F
:102E4000194602223A2300F01DFA3F4B1B684FF04F
:102E5000FF30984771E03D4B1B68FA681A613B4BA5
:102E60001B68FA680832DA60384B1B68BA689A66E1
:102E7000364B1B687A6892B2A3F86620334B1B6806
:102E8000DB68324A1268926E013A120ED2B21A70A0
:102E90002E4B1B68DB6801332C4A1268926E013A94
:102EA000120CD2B21A70294B1B68DB680233274A16
:102EB0001268926E013A120AD2B21A70234B1B6842
:102EC000DB680333214A1268926ED2B2013AD2B261
:102ED0001A701E4B1B68DB6804331C4A1268B2F878
:102EE00066201216D2B21A70184B1B68DB680533C5
:102EF000164A1268B2F866201214D2B21A70134B36
:102F00001B68DB680633114A1268B2F86620120AA1
:102F100092B2D2B21A700D4B1B68DB6807330B4AB2
:102F20001268B2F86620D2B21A70084B1B680822E9
:102F30005A81054B1B68002098471037BD4680BD5D
:102F4000880E0020800E0020840E0020780E0020C5
:102F500080B500AF0548FEF705FA0346002B04D004
:102F600000200021002200F003F880BD712F00082E
:102F700080B584B000AFF860B9607A60FB68002B60
:102F80000FD13E4B1A683E4B1B7810461946022261
:102F90003A2300F077F93B4B1B684FF0FF3098471E
:102FA00068E0394B1B68FA681A61374B1B68FA688E
:102FB0000832DA60344B1B68DB6800221A70324B2F
:102FC0001B68DB68013300221A702F4B1B68DB681B
:102FD000023300221A702C4B1B68DB680333082273
:102FE0001A70294B1B68DB680433BA68013A120E69
:102FF000D2B21A70244B1B68DB680533BA68013AF9
:10300000120CD2B21A70204B1B68DB680633BA6808
:10301000013A120AD2B21A701B4B1B68DB680733E5
:10302000BA68D2B2013AD2B21A70174B1B68DB6889
:10303000083302221A70144B1B68DB6809337A6864
:10304000120CD2B21A70104B1B68DB680A337A6814
:10305000120AD2B21A700C4B1B68DB680B337A6809
:10306000D2B21A70084B1B680C225A81054B1B68A0
:10307000002098471037BD4680BD00BF880E002055
:10308000800E0020840E0020780E002080B582B0D3
:1030900000AF0823FB80FDF77BFD3860114B1B68F8
:1030A0003A681A610F4B1B683A680832DA600D4BB8
:1030B0001B68FA885A810BE0FB88013BFB80094BB7
:1030C0001B68DA68FB881344FA8807498A5C1A701F
:1030D000FB88002BF0D1054B1B6800209847083770
:1030E000BD4680BD780E0020C0B20008840E0020CE
:1030F00080B582B000AF0823FB80FDF749FD386042
:10310000114B1B683A681A610F4B1B683A6808320A
:10311000DA600D4B1B68FA885A810BE0FB88013B93
:10312000FB80094B1B68DA68FB881344FA8807495F
:103130008A5C1A70FB88002BF0D1054B1B680020BD
:1031400098470837BD4680BD780E0020C8B20008F9
:10315000840E002080B582B000AFFDF719FD386005
:10316000454B1B683A681A61434B1B683A68083242
:10317000DA600023FB7109E03F4B1B68DA68FB79DA
:10318000134400221A70FB790133FB71FB79112B78
:10319000F2D9394B1B68DB6870221A70364B1B68FA
:1031A000DB6807330C221A70334B1B6893F86420DA
:1031B000314B1B6893F865309A4244D02E4B1B6804
:1031C000DB689A1C2C4B19682B4B1B6893F86430F6
:1031D0000833DB000B441B79DBB21370264B1B68F2
:1031E000DB6803F10C02244B1968234B1B6893F82E
:1031F00064300833DB000B445B7ADBB213701E4B88
:103200001B68DB6803F10D021B4B19681A4B1B6826
:1032100093F864300833DB000B441B7ADBB2137085
:10322000154B1B6893F864200132D2B283F86420F6
:10323000114B1B6893F86430042B04D10E4B1B68B0
:10324000002283F864200C4B1B6812225A810B4B1E
:103250001B6804331B78122B07D8074B1B68074ADF
:1032600012680432127892B25A81054B1B68002012
:1032700098470837BD4680BD780E00207C0E0020A0
:10328000840E002080B485B000AF786008461146F7
:103290001A460346FB700B46BB7013467B707B6877
:1032A000D3F81832FB60FB6893F86530B978FA6898
:1032B0000833DB0013440A461A71FB6893F8653043
:1032C00018467B781B021946FA6800F10803DB00F8
:1032D00013449960FB6893F865300133DAB2FB68F8
:1032E00083F86520FB6893F86530042B03D1FB68F5
:1032F000002283F865201437BD465DF8047B7047D3
:1033000080B500AF044B1B6800225A81034B1B6839
:103310000020984780BD00BF780E0020840E00205A
:1033200080B582B002AF5A4B1B681B7A002B40F06D
:10333000A280574B1B6893F82030DBB25BB2002BA6
:1033400011DB544B1A68524B1B6893F8213010461E
:10335000194605222023FFF795FF4F4B1B684FF0BE
:10336000FF30984791E04A4B1B684C4A1268023282
:1033700012781106494A1268033212781204114376
:10338000464A12680432127812020A434349096815
:10339000053109780A43DA663D4B1B683F4A1268DB
:1033A00007321278120291B23C4A1268083212783F
:1033B00092B20A4392B292B2A3F87020344B1B68C7
:1033C000DA6E334B1B68B3F870301046194600F0C4
:1033D000B9FA0346002B11DA2E4B1A682C4B1B68E6
:1033E00093F821301046194605222023FFF74AFFA3
:1033F000294B1B684FF0FF30984746E0244B1B6871
:10340000DB69234A1268B2F870201146204A12681C
:10341000B2F8662002FB01F2934211D01D4B1A68EC
:103420001B4B1B6893F821301046194605222023B8
:10343000FFF728FF184B1B684FF0FF30984724E038
:10344000134B1B68DB6E1A464FF0000310490968E6
:10345000B1F8701008460E490968C96900900191D9
:103460000F48FDF7E5FF0346002B03D0012000F0D5
:103470001BF80AE009E00B48FEF72AF80346002B88
:1034800003D00020002100F043F8BD4680BD00BFFE
:10349000780E0020880E0020840E00207C0E002074
:1034A000A93400081135000880B582B000AF03468A
:1034B000FB71FB79002B0FD0104B1A68104B1B7857
:1034C0001046194602223A23FFF7DCFE0D4B1B681B
:1034D0004FF0FF3098470DE00B4B1B6802221A7229
:1034E0000A48FDF7F5FF0346002B03D0002000211A
:1034F00000F00EF80837BD4680BD00BF880E0020E2
:10350000800E0020840E0020780E00201135000867
:1035100080B582B000AF78600B467B807B68002B63
:103520000FD1204B1A68204B1B78104619460422F5
:103530001123FFF7A7FE1D4B1B684FF0FF30984784
:103540002DE01B4B1B681B69002B00D0FEE7184BBE
:103550001B687A681A61164B1B687A680832DA6051
:10356000104B1968124B1B68DA687B88084681216A
:10357000FDF7DCF80E4B1B680D4A1268D16B7A8898
:103580008A1ADA630A4B1B68DB6B002B03D1084BEA
:103590001B6803221A72054B1B68002098470837E6
:1035A000BD4680BD880E0020800E0020840E0020C5
:1035B000780E002080B584B002AF7B4B1B681B7A6D
:1035C000002B40F09D80784B1B6893F82030DBB2D5
:1035D0005BB2002B11DA754B1A68734B1B6893F8BA
:1035E00021301046194605222023FFF74BFE704B71
:1035F0001B684FF0FF309847D2E06B4B1B686D4A59
:1036000012680232127811066A4A1268033212787E
:1036100012041143674A12680432127812020A43F4
:1036200064490968053109780A43DA665E4B1B680C
:10363000604A126807321278120291B25D4A12682B
:103640000832127892B20A4392B292B2A3F8702072
:10365000554B1B68DA6E544B1B68B3F8703010463C
:10366000194600F06FF90346002B11DA4F4B1A6828
:103670004D4B1B6893F82130104619460522202334
:10368000FFF700FE4A4B1B684FF0FF30984787E07A
:10369000454B1B68DB69444A1268B2F8702011463A
:1036A000414A1268B2F8662002FB01F2934211D03F
:1036B0003E4B1A683C4B1B6893F821301046194664
:1036C00005222023FFF7DEFD394B1B684FF0FF304A
:1036D000984765E0344B1B68DB6E1A464FF00003D9
:1036E00031490968B1F8701000913348FDF782FF45
:1036F0000346002B03D0012000F064F850E04FE0B7
:10370000294B1B68DB6BB3F5007F28BF4FF40073B8
:103710007B60254B1B681B6918467968FDF7E0FF45
:103720000346002B0FD0214B1A68244B1B78104600
:10373000194604220323FFF7A5FD1D4B1B684FF01C
:10374000FF3098472CE0184B1B68174A1268D16B62
:103750007A688A1ADA63144B1B68DB6B002B0AD178
:10376000124B1B681846002100F0C0FA104B1B6872
:103770000020984714E01248FDF7CAF90346002BD1
:103780000ED00A4B1A680D4B1B78104619460222C0
:103790003A23FFF777FD064B1B684FF0FF30984741
:1037A0000837BD4680BD00BF780E0020880E00207F
:1037B000840E00207C0E0020C5370008800E0020FB
:1037C0006938000880B582B000AF0346FB71FB7911
:1037D000022B0FD11F4B1A681F4B1B78104619463E
:1037E00002222723FFF74EFD1C4B1B684FF0FF30D2
:1037F00098472BE0FB79002B0FD0164B1A68164B1D
:103800001B781046194602223A23FFF73BFD134B63
:103810001B684FF0FF30984718E0114B1B680122DE
:103820001A721048FDF774F90346002B0ED0094BAD
:103830001A68094B1B781046194602223A23FFF7F3
:1038400021FD064B1B684FF0FF3098470837BD46F7
:1038500080BD00BF880E0020800E0020840E002056
:10386000780E00206938000880B582B000AF78601B
:10387000104B1B687A681A610E4B1B687A68083215
:10388000DA600D4B19680B4B1B68DA68094B1B6833
:10389000DB6BB3F5007F28BF4FF400739BB2084683
:1038A0000121FCF75DFF054B1B6800209847083796
:1038B000BD4680BD780E0020880E0020840E0020BA
:1038C00080B500AF1A4B1B6801331B7803F002036D
:1038D000002B0FD0174B1A68174B1B781046194650
:1038E00005222423FFF7CEFC144B1B684FF0FF305A
:1038F00098471BE0124B1B68DA6E114B1B68B3F83C
:1039000070301046194600F01DF80346002B05DA0A
:103910000A4B1B684FF0FF30984707E0084B1B68C5
:1039200000225A81054B1B680020984780BD00BFCC
:103930007C0E0020880E0020800E0020840E0020C7
:10394000780E002080B582B000AF78600B467B8097
:103950000F4B1B689A6E7B689A4207D37A887B6804
:103960001A440B4B1B689B6E9A420BD9094B1A6881
:10397000094B1B781046194605222123FFF782FCCC
:10398000FF2300E000235BB218460837BD4680BD28
:10399000780E0020880E0020800E002080B584B0B4
:1039A00000AF78607B68D3F81832FB60FB680022B8
:1039B0001A72FB6800225A72FB68002283F86520A5
:1039C000FB68002283F8642078680121FCF732FE4E
:1039D00078688121FCF72EFEFB681433786801219A
:1039E0001A461F23FCF7BCFE1037BD4680BD00BF42
:1039F00080B584B000AF78607B68D3F81832FB6084
:103A0000FB6800221A72FB6801225A72FB681433A9
:103A1000786801211A461F23FCF7A2FE1037BD4625
:103A200080BD00BF80B485B000AF78607B68D3F8FC
:103A30001832FB60FB6800221A721437BD465DF82D
:103A4000047B704780B584B000AF78600B46FB7094
:103A50007B68D3F81832FB60FB681B7A022B04D01A
:103A6000022B16DB042B14DC0EE00C4A7B6813607F
:103A7000FB6893F82120FB682333786811461A46C7
:103A8000074BFEF7EDFF05E07868002100F02EF906
:103A900000E000BF1037BD4680BD00BF8C0E002087
:103AA000A53A000880B582B000AF0346FB7197F9D4
:103AB0000730002B05DA044B1B681846012100F083
:103AC00015F90837BD4680BD8C0E002080B584B046
:103AD00000AF78600B46FB707B68D3F81832FB6050
:103AE000FB681B7A002B02D0012B04D012E078680F
:103AF00000F02CF80EE0094A7B681360FB6893F82D
:103B00002120FB682333786811461A46044BFEF7E0
:103B1000A7FF00BF1037BD4680BD00BF8C0E002040
:103B2000253B000880B582B000AF0346FB7197F9D2
:103B30000730002B05DA044B1B681846012100F002
:103B4000D5F80837BD4680BD8C0E002080B584B006
:103B500000AF78607B68D3F81832FB60FB689A6925
:103B6000FB689A63FB68DA69FB68DA6378680121AD
:103B7000FCF710FE03461F2B13D1FB685B691B4A41
:103B800093420ED1FB6893F82130012B09D8FB68D2
:103B900093F82230002B04D0FB6893F82230102BCE
:103BA0000FD9FB6893F82130786819460522202345
:103BB000FFF768FBFB6802225A72786800F0C0F8D1
:103BC00010E00B4A7B6813600A4AFB681360FB68CD
:103BD00093F82120FB682333786811461A46064B78
:103BE000FEF73EFF1037BD4680BD00BF5553424330
:103BF0008C0E0020900E0020FD3B000880B582B0A6
:103C000000AF0346FB7197F90730002B11DA214B07
:103C10001B681B7A052B06D11F4B1B681846012118
:103C200000F064F832E01C4B1B68184600F088F87E
:103C30002CE0184B1B681B7A022B27D0154B1B68F6
:103C40001B7A012B22D0134B1B681B7A032B1DD030
:103C5000104B1B685B89002B0DD00F4B19680D4B67
:103C60001B68DA680B4B1B685B89084611461A46CD
:103C700000F014F80AE0074B1B685B89002B05D1A4
:103C8000054B1B681846002100F030F80837BD4688
:103C900080BD00BF900E00208C0E002080B586B045
:103CA00000AFF860B9601346FB80FB68D3F81832A8
:103CB0007B61FA887B69DB69934228BF1346FB80EE
:103CC0007B69DA6BFB88D21A7B69DA637B69002235
:103CD00083F840207B6904221A72FB88F8688121EE
:103CE000BA68FCF723FD1837BD4680BD80B584B0A7
:103CF00000AF78600B46FB707B68D3F81832FB602E
:103D0000FB680E4A5A63FB68FA7883F84020FB6828
:103D100000221A72FB683433786881211A460D2319
:103D2000FCF704FDFB681433786801211A461F2351
:103D3000FCF716FD1037BD4680BD00BF55534253FA
:103D400080B584B000AF78607B68D3F81832FB6030
:103D5000FB6893F82030002B0BD1FB68DB69002B4C
:103D600007D0FB685B7A002B03D178680121FCF750
:103D700075FC78688121FCF771FCFB685B7A022B8B
:103D800007D1FB681433786801211A461F23FCF71A
:103D9000E7FC1037BD4680BD80B584B000AF7860C9
:103DA0000B46FB707B68D3F81832FB60FB685B7ACC
:103DB000022B07D178688121FCF750FCFB680022B8
:103DC0005A720BE0FB785BB2002B07DAFB685B7A78
:103DD000012B03D078680121FFF788FF1037BD461B
:103DE00080BD00BF80B584B000AF78600B46FB702B
:103DF0000023FB817B681B7C002B0ED1786801219E
:103E000002224FF40073FCF7E7FB7868812102225D
:103E10004FF40073FCF7E0FB0BE07868012102220D
:103E20004023FCF7D9FB7868812102224023FCF76C
:103E3000D3FB742007F03CF903461A467B68C3F8AD
:103E400018227B68D3F81832002B02D10123FB81A2
:103E500009E07868FFF7A2FD7B68D3F818320022EA
:103E60001A610023FB81FB89DBB218461037BD467F
:103E700080BD00BF80B582B000AF78600B46FB709C
:103E800078680121FCF7C2FB78688121FCF7BEFB52
:103E90007868FFF7C7FD7B68D3F81832002B09D08C
:103EA0007B68D3F81832184607F00AF97B680022BD
:103EB000C3F81822002318460837BD4680BD00BF4E
:103EC00080B584B000AF786039607B68D3F8183271
:103ED000FB603B681B7803F06003002B46D0202B6F
:103EE00000D09DE03B685B78FE2B02D0FF2B1ED0FC
:103EF00035E03B685B88002B13D13B68DB88012BE6
:103F00000FD13B681B78DBB25BB2002B09DAFB6890
:103F100000221A60FB68786819460122FDF726FE28
:103F200023E078683968FEF783FA022379E03B687A
:103F30005B88002B0DD13B68DB88002B09D13B68E7
:103F40001B78DBB25BB2002B03DB7868FFF750FD18
:103F50000BE078683968FEF76BFA022361E0786855
:103F60003968FEF765FA02235BE059E03B685B784D
:103F70000A2B04D00B2B0AD0012B0FD04FE0FB688B
:103F80000433786819460122FDF7F0FD47E03B68ED
:103F90005B88DBB21A46FB685A6040E03B689B884E
:103FA000DBB278681946FCF745FB3B689B88DBB2BF
:103FB00078681946FCF72AFB3B689B88DBB25BB24A
:103FC000002B12DA7B681B7C002B07D178688121DB
:103FD00002224FF40073FCF7FFFA18E078688121A1
:103FE00002224023FCF7F8FA11E07B681B7C002BCF
:103FF00007D17868012102224FF40073FCF7ECFA34
:1040000005E07868012102224023FCF7E5FA3B68CD
:104010009B88DBB278681946FFF7BEFE00BF00BF81
:10402000002318461037BD4680BD00BF80B582B062
:1040300000AF78600B46FB70FB7878681946FFF795
:1040400001FD002318460837BD4680BD80B582B00B
:1040500000AF78600B46FB70FB7878681946FFF775
:1040600035FD002318460837BD4680BD80B582B0B7
:1040700000AF78607B68D3F81832002B11D07B68D2
:10408000D3F818321B69002B0BD07B68D3F8183299
:104090001B691846FCF7B2FD7B68D3F81832002282
:1040A0001A61002318460837BD4680BD80B483B02E
:1040B00000AF78607B6820221A80034B18460C37CB
:1040C000BD465DF8047B70477000002080B483B06B
:1040D00000AF78607B6820221A80034B18460C37AB
:1040E000BD465DF8047B70479000002080B483B02B
:1040F00000AF78607B6820221A80034B18460C378B
:10410000BD465DF8047B7047B000002080B483B0EA
:1041100000AF78607B680A221A80034B18460C3780
:10412000BD465DF8047B7047D000002084B080B5A8
:1041300082B000AF786007F1140080E80E00BB6A1F
:10414000012B20D17B689B6B23F480327B689A63C0
:104150007B68DB6823F4840323F040037A68D36030
:104160007B68DB6823F440127B68DA603B6C012BD0
:1041700005D17B68DB6843F480127B68DA6078687D
:1041800001F0CCF90CE07B68DB6843F040027B680F
:10419000DA60786801F0C2F97B684FF480329A6384
:1041A0003B6A012B0BD17B689B6843F00C027B6858
:1041B0009A607B689B6843F020027B689A600023CA
:1041C00018460837BD46BDE8804004B0704700BFC0
:1041D00080B483B000AF78607B689B6843F00102D5
:1041E0007B689A60002318460C37BD465DF8047B57
:1041F000704700BF80B483B000AF78607B689B6875
:1042000023F001027B689A60002318460C37BD46F4
:104210005DF8047B704700BF80B582B000AF786066
:104220000B46FB707B68DB6823F0C0427B68DA607A
:10423000FB78012B06D17B68DB6843F000527B687A
:10424000DA6008E0FB78002B05D17B68DB6843F07F
:1042500080427B68DA60322006F0BEFE00231846FA
:104260000837BD4680BD00BF84B080B584B000AFC4
:10427000786007F11C0080E80E000023FB607B687B
:104280009B6B43F400227B689A633B6C002B05D147
:104290007B689B6B43F400127B689A637B6803F531
:1042A00060631A46002313607B6803F500631A46B7
:1042B0007B6803F500631B6813603B6B012B0CD11B
:1042C0007B6A002B04D17868002100F041F908E0F6
:1042D0007868012100F03CF903E07868032100F0E0
:1042E00037F97868102100F0EBF8786800F00EF9E3
:1042F0007B6803F500631A46002313617B6803F5AE
:1043000000631A46002353617B6803F500631A4675
:104310004FF0FF3393617B6803F500631A46002377
:10432000D3610023FB6031E0FB685A017B681344D2
:1043300003F510631B68002B0ADAFB685A017B68DF
:10434000134403F510631A464FF09043136008E0DE
:10435000FB685A017B68134403F510631A46002377
:104360001360FB685A017B68134403F510631A4617
:1043700000231361FB685A017B68134403F5106343
:104380001A46FF239360FB680133FB60FA69FB6800
:104390009A42C9D80023FB6031E0FB685A017B6870
:1043A000134403F530631B68002B0ADAFB685A01DB
:1043B0007B68134403F530631A464FF09043136053
:1043C00008E0FB685A017B68134403F530631A4622
:1043D00000231360FB685A017B68134403F53063C4
:1043E0001A4600231361FB685A017B68134403F5E6
:1043F00030631A46FF239360FB680133FB60FA6960
:10440000FB689A42C9D87B6803F500631A467B684B
:1044100003F500631B6923F480731361BB6A012BEE
:1044200017D17B6803F500631A46234B13637B683F
:1044300003F500631A467B6803F500631B6B43F4C6
:10444000803343F0030313637B6803F500631B6B46
:10445000FB607B6800229A617B686FF080425A6142
:10446000BB6A002B05D17B689B6943F010027B6817
:104470009A617B689A69114B13437A6893617B6BED
:10448000002B05D07B689B6943F008027B689A612A
:104490003B6C012B07D17B689B6943F0804343F061
:1044A00004037A689361002318461037BD46BDE8BF
:1044B000804004B0704700BF0001800000383C809D
:1044C00080B485B000AF786039600023FB603B6842
:1044D0009B0143F020027B681A61FB680133FB609B
:1044E000FB68094A934201D9032306E07B681B69F4
:1044F00003F02003002BF0D1002318461437BD46EB
:104500005DF8047B704700BF400D030080B485B0A8
:1045100000AF78600023FB607B6810221A61FB68A3
:104520000133FB60FB68094A934201D9032306E08B
:104530007B681B6903F01003002BF0D100231846A1
:104540001437BD465DF8047B704700BF400D030083
:1045500080B483B000AF78600B46FB707B6803F5D6
:10456000006319467B6803F500631A68FB78134300
:104570000B60002318460C37BD465DF8047B70477E
:1045800080B485B000AF78600023FB737B6803F5CF
:1045900000639B6803F00603002B02D10023FB732A
:1045A0001CE07B6803F500639B6803F00603022BA5
:1045B00007D07B6803F500639B6803F00603062BB6
:1045C00002D10323FB7309E07B6803F500639B685A
:1045D00003F00603042B01D10223FB73FB7B184677
:1045E0001437BD465DF8047B704700BF80B483B0CC
:1045F00000AF786039603B685B78012B3ED17B6807
:1046000003F5006319467B6803F50063DA693B68CC
:104610001B781846012383409BB21343CB613B6850
:104620001B785A017B68134403F510631B6803F47D
:104630000043002B5CD13B681B785A017B68134414
:1046400003F5106318463B681B785A017B681344D6
:1046500003F510631A683B689B68C3F30A03396863
:10466000C97889040B433968097889050B431343DA
:1046700043F0805343F40043036039E07B6803F563
:10468000006319467B6803F50063DB693A681278BA
:1046900010460122824012041343CB613B681B7811
:1046A0005A017B68134403F530631B6803F400432D
:1046B000002B1DD13B681B785A017B68134403F51E
:1046C000306318463B681B785A017B68134403F536
:1046D00030631A683B689B68C3F30A033968C9787A
:1046E00089040B43134343F0805343F400430360B6
:1046F000002318460C37BD465DF8047B704700BFA9
:1047000080B483B000AF786039603B685B78012B80
:1047100035D17B6803F5006319467B6803F50063B8
:10472000DA6B3B681B781846012383409BB2DB435E
:104730001340CB637B6803F5006319467B6803F580
:104740000063DA693B681B781846012383409BB2FB
:10475000DB431340CB613B681B785A017B681344F1
:1047600003F5106319463B681B785A017B681344B4
:1047700003F510631B6823F400430B6034E07B688F
:1047800003F5006319467B6803F50063DA6B3B6849
:104790001B781846012383401B04DB431340CB6383
:1047A0007B6803F5006319467B6803F50063DA69EB
:1047B0003B681B781846012383401B04DB431340EE
:1047C000CB613B681B785A017B68134403F5306367
:1047D00019463B681B785A017B68134403F5306324
:1047E0001B6823F400430B60002318460C37BD46BA
:1047F0005DF8047B704700BF90B589B002AFF860E8
:10480000B9601346FB710023FB82BB685B78012B08
:1048100040F04681BB685B69002B3BD1BB681B78CD
:104820005A01FB68134403F510631946BB681B78F3
:104830005A01FB68134403F510631B6923F0FF530F
:1048400023F4C0130B61BB681B785A01FB68134447
:1048500003F510631946BB681B785A01FB681344C3
:1048600003F510631B6943F400230B61BB681B78DD
:104870005A01FB68134403F510631946BB681B78A3
:104880005A01FB68134403F510631B69DB0CDB045E
:104890000B6186E0BB681B785A01FB68134403F583
:1048A00010631946BB681B785A01FB68134403F573
:1048B00010631B69DB0CDB040B61BB681B785A01BE
:1048C000FB68134403F510631946BB681B785A0153
:1048D000FB68134403F510631B6923F0FF5323F4B3
:1048E000C0130B61BB681B785A01FB68134403F5C6
:1048F00010631846BB681B785A01FB68134403F524
:1049000010631A69BB685969BB689B680B44591EE0
:10491000BB689B68B1FBF3F3D9048C4B0B4013438A
:104920000361BB681B785A01FB68134403F51063ED
:104930001946BB681B785A01FB68134403F51063E2
:104940001A69BB685B69C3F3120313430B61BB684D
:10495000DB78012B25D1BB681B785A01FB68134417
:1049600003F510631946BB681B785A01FB681344B2
:1049700003F510631B6923F0C0430B61BB681B7810
:104980005A01FB68134403F510631946BB681B7892
:104990005A01FB68134403F510631B6943F000538D
:1049A0000B61FB79012B0BD1BB681B785A01FB68AB
:1049B000134403F510631A46BB681B69536116E084
:1049C000BB68DB78012B12D0BB685B69002B0ED073
:1049D000FB6803F500631946FB6803F500635B6B36
:1049E000BA68127810460122824013434B63BB68B9
:1049F000DB78012B2ED1FB6803F500639B6803F481
:104A00008073002B13D1BB681B785A01FB681344D9
:104A100003F510631946BB681B785A01FB68134401
:104A200003F510631B6843F000530B6012E0BB6892
:104A30001B785A01FB68134403F510631946BB68E1
:104A40001B785A01FB68134403F510631B6843F09D
:104A500080530B60BB681B785A01FB68134403F555
:104A600010631946BB681B785A01FB68134403F5B1
:104A700010631B6843F004430B60BB68DB78012BB9
:104A800040F0F580BB68D968BB681A78BB685B6981
:104A90009CB2FB790093F868234600F04DFAE6E0FB
:104AA000BB681B785A01FB68134403F53063194651
:104AB000BB681B785A01FB68134403F530631B691C
:104AC000DB0CDB040B61BB681B785A01FB681344E9
:104AD00003F530631946BB681B785A01FB68134421
:104AE00003F530631B6923F0FF5323F4C0130B61FC
:104AF000BB685B69002B2BD1BB681B785A01FB6834
:104B0000134403F530631946BB681B785A01FB68F0
:104B1000134403F530631A69BB689B68C3F312033F
:104B200013430B61BB681B785A01FB68134403F500
:104B300030631946BB681B785A01FB68134403F5C0
:104B400030631B6943F400230B613CE00000F81F55
:104B5000BB685A69BB689B6813445A1EBB689B6854
:104B6000B2FBF3F3FB82BB681B785A01FB6813446A
:104B700003F530631946BB681B785A01FB68134480
:104B800003F530631A69FB8ADB0418463A4B03408D
:104B900013430B61BB681B785A01FB68134403F590
:104BA00030631846BB681B785A01FB68134403F551
:104BB00030631A69BB689B68F98A01FB03F3C3F38E
:104BC000120313430361FB79012B0AD1BB681B78E5
:104BD0005A01FB68134403F530631A46BB68DB686F
:104BE0005361BB68DB78012B2ED1FB6803F50063B2
:104BF0009B6803F48073002B13D1BB681B785A01A8
:104C0000FB68134403F530631946BB681B785A01EF
:104C1000FB68134403F530631B6843F000530B60DB
:104C200012E0BB681B785A01FB68134403F530633C
:104C30001946BB681B785A01FB68134403F53063BF
:104C40001B6843F080530B60BB681B785A01FB68FC
:104C5000134403F530631946BB681B785A01FB689F
:104C6000134403F530631B6843F004430B600023D7
:104C700018461C37BD4690BD0000F81F80B485B0B3
:104C800000AFF860B9601346FB71BB685B78012B1D
:104C900040F0D180BB685B69002B3BD1BB681B78BF
:104CA0005A01FB68134403F510631946BB681B786F
:104CB0005A01FB68134403F510631B6923F0FF538B
:104CC00023F4C0130B61BB681B785A01FB681344C3
:104CD00003F510631946BB681B785A01FB6813443F
:104CE00003F510631B6943F400230B61BB681B7859
:104CF0005A01FB68134403F510631946BB681B781F
:104D00005A01FB68134403F510631B69DB0CDB04D9
:104D10000B615AE0BB681B785A01FB68134403F52A
:104D200010631946BB681B785A01FB68134403F5EE
:104D300010631B69DB0CDB040B61BB681B785A0139
:104D4000FB68134403F510631946BB681B785A01CE
:104D5000FB68134403F510631B6923F0FF5323F42E
:104D6000C0130B61BB685A69BB689B689A4203D940
:104D7000BB689A68BB685A61BB681B785A01FB68BC
:104D8000134403F510631946BB681B785A01FB688E
:104D9000134403F510631B6943F400230B61BB68E4
:104DA0001B785A01FB68134403F510631946BB686E
:104DB0001B785A01FB68134403F510631A69BB683A
:104DC0005B69C3F3120313430B61FB79012B0BD116
:104DD000BB681B785A01FB68134403F510631A463D
:104DE000BB681B69536112E0BB685B69002B0ED086
:104DF000FB6803F500631946FB6803F500635B6B12
:104E0000BA68127810460122824013434B63BB6894
:104E10001B785A01FB68134403F510631946BB68FD
:104E20001B785A01FB68134403F510631B6843F0B9
:104E300004430B6079E0BB681B785A01FB6813449C
:104E400003F530631946BB681B785A01FB681344AD
:104E500003F530631B69DB0CDB040B61BB681B785B
:104E60005A01FB68134403F530631946BB681B788D
:104E70005A01FB68134403F530631B6923F0FF53A9
:104E800023F4C0130B61BB685B69002B03D0BB68C4
:104E90009A68BB685A61BB681B785A01FB68134467
:104EA00003F530631946BB681B785A01FB6813444D
:104EB00003F530631B6943F400230B61BB681B7867
:104EC0005A01FB68134403F530631946BB681B782D
:104ED0005A01FB68134403F530631A69BB689B6889
:104EE000C3F3120313430B61FB79012B0AD1BB6897
:104EF0001B785A01FB68134403F530631A46BB68FC
:104F0000DB685361BB681B785A01FB68134403F5E7
:104F100030631946BB681B785A01FB68134403F5DC
:104F200030631B6843F004430B60002318461437BA
:104F3000BD465DF8047B704780B487B000AFF86071
:104F4000B96011461A460B46FB711346BB8000231D
:104F50003B6100237B6197F82030002B1DD1BB887B
:104F60000333002B00DA03339B103B6100237B618A
:104F70000FE0FB791A03FB68134403F580531A46CC
:104F8000BB681B6813607B6901337B61BB680433BA
:104F9000BB607A693B699A42EBD3002318461C3701
:104FA000BD465DF8047B704780B487B000AFF86001
:104FB000B9601346FB8000237B61FB880333002B21
:104FC00000DA03339B103B6100237B610BE0FB683D
:104FD00003F580531A68BB681A607B6901337B61F3
:104FE000BB680433BB607A693B699A42EFD3BB6804
:104FF00018461C37BD465DF8047B704780B483B00B
:1050000000AF786039603B685B78012B30D13B683A
:105010001B785A017B68134403F510631B68002B4F
:1050200012DB3B681B785A017B68134403F510635D
:1050300019463B681B785A017B68134403F51063DB
:105040001B6823F080430B603B681B785A017B6828
:10505000134403F5106319463B681B785A017B68BB
:10506000134403F510631B6843F400130B602FE037
:105070003B681B785A017B68134403F530631B6857
:10508000002B12DB3B681B785A017B68134403F545
:10509000306319463B681B785A017B68134403F55B
:1050A00030631B6823F080430B603B681B785A0118
:1050B0007B68134403F5306319463B681B785A013B
:1050C0007B68134403F530631B6843F400130B60E3
:1050D000002318460C37BD465DF8047B704700BFBF
:1050E00080B483B000AF786039603B685B78012B97
:1050F0002ED13B681B785A017B68134403F510637B
:1051000019463B681B785A017B68134403F510630A
:105110001B6823F400130B603B68DB78032B03D080
:105120003B68DB78022B41D13B681B785A017B68D6
:10513000134403F5106319463B681B785A017B68DA
:10514000134403F510631B6843F080530B602DE09C
:105150003B681B785A017B68134403F5306319469A
:105160003B681B785A017B68134403F530631B6866
:1051700023F400130B603B68DB78032B03D03B6800
:10518000DB78022B12D13B681B785A017B681344F1
:1051900003F5306319463B681B785A017B6813445A
:1051A00003F530631B6843F080530B6000231846FF
:1051B0000C37BD465DF8047B704700BF80B584B0F6
:1051C00000AF78600023FB6014E0FB685A017B6845
:1051D000134403F510631A46FF239360FB685A01DA
:1051E0007B68134403F530631A46FF239360FB6822
:1051F0000133FB60FB680E2BE7D97B6803F5006386
:105200001A464FF0FF3393617B6803F500631A463B
:10521000002313617B6803F500631A460023536182
:105220007B6803F500631A460023D3617868FFF7B3
:105230006DF978681021FFF743F9002318461037FD
:10524000BD4680BD80B483B000AF78600B46FB7074
:105250007B6803F500631A467B6803F500631B68EF
:1052600023F4FE6313607B6803F5006319467B68D3
:1052700003F500631A68FB781B0103F4FE63134314
:105280000B60002318460C37BD465DF8047B704761
:1052900080B582B000AF78607B6803F500631A4682
:1052A0007B6803F500635B6823F00203536003200F
:1052B00005F092FE002318460837BD4680BD00BFAA
:1052C00080B582B000AF78607B6803F500631A4652
:1052D0007B6803F500635B6843F0020353600320BF
:1052E00005F07AFE002318460837BD4680BD00BF92
:1052F00080B485B000AF78600023FB607B685B6999
:10530000FB607B689B69FA681340FB60FB6818468A
:105310001437BD465DF8047B704700BF80B485B08C
:1053200000AF78607B6803F500639B69FB607B6876
:1053300003F50063DB69FA681340FB60FB681B0C34
:1053400018461437BD465DF8047B704780B485B0BD
:1053500000AF78607B6803F500639B69FB607B6846
:1053600003F50063DB69FA681340FB60FB689BB2DE
:1053700018461437BD465DF8047B704780B485B08D
:1053800000AF78600B46FB70FB785A017B681344D2
:1053900003F530639B68FB607B6803F500635B6922
:1053A000FA681340FB60FB6818461437BD465DF889
:1053B000047B704780B487B000AF78600B46FB7009
:1053C0007B6803F500631B697B617B6803F5006301
:1053D0005B6B3B61FB783A6922FA03F3DB01DBB2DA
:1053E0007A6913437B61FB785A017B68134403F5A8
:1053F00010639A687B691340FB60FB6818461C3792
:10540000BD465DF8047B704780B483B000AF786020
:105410007B685B6903F0010318460C37BD465DF8F5
:10542000047B704780B483B000AF78607B6803F57D
:1054300010631A467B6803F510631B6823F4FF634F
:1054400023F0070313607B6803F500639B6803F098
:105450000603042B0AD17B6803F510631A467B68A8
:1054600003F510631B6843F0030313607B6803F5C7
:1054700000631A467B6803F500635B6843F480733E
:105480005360002318460C37BD465DF8047B704717
:1054900080B485B000AFF8600B467A60FB72FB68A1
:1054A00003F530631A4600231361FB6803F530638C
:1054B0001A46FB6803F530631B6943F4002313614C
:1054C000FB6803F530631A46FB6803F530631B691C
:1054D00043F018031361FB6803F530631A46FB6859
:1054E00003F530631B6943F0C0431361FB7A012B62
:1054F0000CD1FB6803F530631A467B685361FB6887
:1055000003F530631A464FF08023136000231846DA
:105510001437BD465DF8047B704700BF80B485B08A
:1055200000AF78600023FB60FB680133FB60FB6821
:10553000134A934201D903231BE07B681B69002BAC
:10554000F2DA0023FB607B681B6943F001027B6891
:105550001A61FB680133FB60FB68094A934201D979
:10556000032306E07B681B6903F00103002BF0D1E5
:10557000002318461437BD465DF8047B704700BF12
:10558000400D030080B582B000AF78607B68002BCF
:1055900001D1012357E07B6893F85130DBB2002B37
:1055A00006D17B68002283F850207868FCF71AFA4D
:1055B0007B68022283F851207B681B687A68126836
:1055C000126822F040021A607B681B687A68516892
:1055D0007A68926811437A68D26811437A681269CE
:1055E00011437A68526911437A68926902F4007231
:1055F00011437A68D26911437A68126A11437A6852
:10560000926A0A431A607B681B687A689269120C76
:1056100002F004017A68526A0A435A607B681B6888
:105620007A68D26A1A617B681B687A681268D269E4
:1056300022F40062DA617B6800225A657B680122ED
:1056400083F85120002318460837BD4680BD00BFAF
:1056500090B587B000AFF860B9607A607B800023B6
:105660007B61FB6893F85130DBB27B617B69012B76
:105670000ED0FB685B68B3F5827F40F0CA80FB68A0
:105680009B68002B40F0C5807B69222B40F0C180D5
:10569000BB68002B05D07B68002B02D07B88002BD9
:1056A00001D10123B6E0FB6893F85030012B01D102
:1056B0000223AFE0FB68012283F85020FB6893F8D7
:1056C0005130DBB2222B03D0FB68322283F8512009
:1056D000FB6800225A65FB68BA681A63FB687A881F
:1056E0009A86FB687A88DA86FB687A689A63FB6830
:1056F0007A889A87FB687A88DA87FB6800229A643E
:10570000FB680022DA64FB689B6AB3F5005F0FD187
:10571000FB681B68FA681268126822F400521A606B
:10572000FB681B68FA681268126842F400521A603B
:10573000FB6893F85130DBB2222B08D1FB685B6C1D
:10574000364A1A64FB685B6C354ADA6307E0FB682B
:105750005B6C344A1A64FB685B6C334ADA63FB683F
:105760005B6C324A9A64FB685A6CFB681B680C33AA
:105770001946FB689B6B1C46FB68DB8F1046224674
:1057800002F0CAF8FB681B68FA681268526842F0B7
:1057900001025A60FB681B6C0022DA63FB6893F815
:1057A0005130DBB2322B04D1FB681B6C1F4A9A6468
:1057B00003E0FB681B6C00229A64FB681A6CFB68B0
:1057C0001B6B1946FB681B680C331C46FB68DB8EA1
:1057D0001046224602F0A0F8FB68002283F8502011
:1057E000FB681B681B6803F04003002B07D1FB68B4
:1057F0001B68FA681268126842F040021A60FB687F
:105800001B68FA681268526842F002025A6000236C
:1058100000E0022318461C37BD4690BD955A00088B
:1058200059580008B15A0008455A0008CD5A0008D6
:1058300080B483B000AF78600C37BD465DF8047B60
:10584000704700BF80B483B000AF78600C37BD46AE
:105850005DF8047B704700BF80B584B000AF78600E
:105860007B689B6BFB607B681B681B6803F4807321
:10587000002B79D1FB689B68002B08D1FB685B6823
:10588000B3F5827F03D1F86800F074F85CE0FB6840
:105890005B68B3F5827F11D1FB689B68B3F5004F5D
:1058A00004D0FB689B68B3F5806F07D1FB681B6869
:1058B000FA681268126822F040021A60FB681B68DE
:1058C000FA681268526822F001025A60FB680022EE
:1058D000DA87FB689B6AB3F5005F35D1F868012170
:1058E00000220A2300F010F90346002B05D0FB68C4
:1058F0005B6D43F02002FB685A65FB681B68DB6840
:105900009BB27B817B89F868012101220A2300F088
:10591000FBF80346002B05D0FB685B6D43F02002CB
:10592000FB685A65FB681B689B6803F01003002B3B
:105930000AD0FB685B6D43F00202FB685A65FB68A6
:105940001B686FF010029A60FB68012283F85120F7
:10595000FB685B6D002B03D0F868FBF789FC06E061
:10596000F868FBF769FC02E0F868FBF765FC1037A4
:10597000BD4680BD80B584B000AF78607B689B6A0F
:10598000B3F5005F26D17868012100220A2300F0D8
:10599000BBF80346002B05D07B685B6D43F020020B
:1059A0007B685A657B681B68DB689BB2FB81FB895F
:1059B0007B681B689B6803F01003002B0AD07B6890
:1059C0005B6D43F002027B685A657B681B686FF071
:1059D00010029A607868022100220A2300F094F8ED
:1059E0000346002B05D07B685B6D43F020027B688B
:1059F0005A657B681B687A681268526822F0020256
:105A00005A607868802101220A2300F07DF803465D
:105A1000002B05D07B685B6D43F020027B685A65E4
:105A20007B681B687A681268526822F001025A602B
:105A30007B680022DA867B680022DA871037BD4651
:105A400080BD00BF80B584B000AF78607B689B6B81
:105A5000FB607B681B681B6803F48073002B12D10A
:105A6000F868FFF787FFFB68012283F85120FB6885
:105A70005B6D002B03D0F868FBF7FAFB06E0F868D3
:105A8000FBF776F902E0F868FBF772F91037BD46CC
:105A900080BD00BF80B584B000AF78607B689B6B31
:105AA000FB60F868FFF7C4FE1037BD4680BD00BF3D
:105AB00080B584B000AF78607B689B6BFB60F86852
:105AC000FFF7C0FE1037BD4680BD00BF80B584B073
:105AD00000AF78607B689B6BFB60FB680022DA8616
:105AE000FB680022DA87FB68012283F85120FB68FB
:105AF0005B6D43F01002FB685A65F868FBF7B8FB72
:105B00001037BD4680BD00BF80B586B000AFF860DD
:105B1000B9603B601346FB7100237B6105F050FACE
:105B20007861FB79002B47D13DE03B68B3F1FF3F43
:105B300039D03B68002B07D005F042FA02467B695A
:105B4000D21A3B689A422ED9FB681B68FA68126821
:105B5000526822F0E0025A60FB681B68FA6812681B
:105B6000126822F040021A60FB689B6AB3F5005F7E
:105B70000FD1FB681B68FA681268126822F40052A1
:105B80001A60FB681B68FA681268126842F40052D7
:105B90001A60FB68012283F85120FB68002283F819
:105BA0005020032350E0FB681B689A68BB681A40CA
:105BB000BB689A42B9D146E03DE03B68B3F1FF3F94
:105BC00039D03B68002B07D005F0FAF902467B6913
:105BD000D21A3B689A422ED9FB681B68FA68126891
:105BE000526822F0E0025A60FB681B68FA6812688B
:105BF000126822F040021A60FB689B6AB3F5005FEE
:105C00000FD1FB681B68FA681268126822F4005210
:105C10001A60FB681B68FA681268126842F4005246
:105C20001A60FB68012283F85120FB68002283F888
:105C30005020032308E0FB681B689A68BB681A4081
:105C4000BB689A42B9D0002318461837BD4680BDBC
:105C500080B594B000AF78600023FB647B681B685C
:105C600003F00103002B47D09D4B9B6803F00C030E
:105C7000042B0BD09A4B9B6803F00C03082B07D125
:105C8000974B5B6803F48003002B01D00123BBE139
:105C9000944B00221A7005F093F9F86409E005F0BE
:105CA0008FF90246FB6CD31AB3F5FA7F01D90323AF
:105CB000AAE18B4B1B6803F40033002BEFD1894A18
:105CC0007B685B68DBB213707B685B68002B13D06A
:105CD00005F076F9F86409E005F072F90246FB6C0C
:105CE000D31AB3F5FA7F01D903238DE17C4B1B68EE
:105CF00003F40033002BEFD07B681B6803F0020332
:105D0000002B61D0764B9B6803F00C03002B0BD06B
:105D1000734B9B6803F00C03082B0CD1704B5B6832
:105D200003F48003002B06D17B68DB68012B01D0D4
:105D3000012369E130E07B68DB68002B16D06A4BF9
:105D400001221A6005F03CF9F86408E005F038F922
:105D50000246FB6CD31A642B01D9032354E1604B38
:105D60001B6803F00203002BF0D015E05E4B00220D
:105D70001A6005F025F9F86408E005F021F90246FB
:105D8000FB6CD31A642B01D903233DE1544B1B68F0
:105D900003F00203002BF0D15148514B1B6823F054
:105DA000F8027B681B69F821B964B96C91FAA1F11A
:105DB0007964796C3964396CB1FA81F1F963F96B02
:105DC000C9B28B40134303607B681B6803F0080370
:105DD000002B30D07B685B69002B16D0434B01222F
:105DE0001A6005F0EDF8F86408E005F0E9F80246FD
:105DF000FB6CD31A642B01D9032305E1384B5B6F8D
:105E000003F00203002BF0D015E0384B00221A609B
:105E100005F0D6F8F86408E005F0D2F80246FB6C0D
:105E2000D31A642B01D90323EEE02D4B5B6F03F0F3
:105E30000203002BF0D17B681B6803F00403002BE6
:105E400060D0274A264B1B6C43F080531364284ACA
:105E5000274B1B6843F48073136005F0B1F8F864B6
:105E600008E005F0ADF80246FB6CD31A642B01D9AB
:105E70000323C9E01E4B1B6803F48073002BF0D092
:105E80001C4B00221A7005F09BF8F8640AE005F03C
:105E900097F80246FB6CD31A41F28832934201D93B
:105EA0000323B1E00E4B1B6F03F00203002BEED176
:105EB000104A7B689B68DBB213707B689B68002B81
:105EC00020D005F07DF8F86416E005F079F8024678
:105ED000FB6CD31A41F2883293420DD9032393E02D
:105EE000003802400238024000004742800E47421C
:105EF0000070004070380240454B1B6F03F00203F6
:105F0000002BE2D07B689B69002B7CD0404B9B68C8
:105F100003F00C03082B74D03E4B00221A6005F0EE
:105F20004FF8F86408E005F04BF80246FB6CD31A12
:105F3000642B01D9032367E0354B1B6803F0007322
:105F4000002BF0D17B689B69022B5CD130487B68C9
:105F50001A6A7B685B6A47F6C071B963B96B91FADC
:105F6000A1F17963796B3963396BB1FA81F1F96227
:105F7000F96AC9B28B401A437B689B6A5B08013B94
:105F80004FF44031B962B96A91FAA1F17962796A44
:105F90003962396AB1FA81F1F961F969C9B28B40A4
:105FA0001A437B68DB691A437B68DB6A4FF07061D8
:105FB000B961B96991FAA1F1796179693961396990
:105FC000B1FA81F1F960F968C9B28B40134343F02B
:105FD000005343600F4B01221A6004F0F1FFF86494
:105FE00008E004F0EDFF0246FB6CD31A642B01D9E4
:105FF000032309E0064B1B6803F00073002BF0D06D
:1060000001E0012300E0002318465037BD4680BD63
:10601000003802406000474280B584B000AF78602D
:1060200039600023FB60A64B1B6803F00F023B683E
:106030009A4280F09080A24B3A68D2B21A70A04B7C
:106040001B6803F00F023B689A4201D0012333E141
:106050007B681B6803F00203002B08D09949994B19
:106060009B6823F0F0027B689B6813438B607B681E
:106070001B6803F00103002B00F0FB807B685B686A
:10608000012B07D18F4B1B6803F40033002B15D174
:10609000012311E17B685B68022B07D1894B1B68E8
:1060A00003F00073002B09D1012305E1854B1B6828
:1060B00003F00203002B01D10123FDE08149814B54
:1060C0009B6823F003027B685B6813438B6004F0DA
:1060D00077FFF8607B685B68012B12D10AE004F05F
:1060E0006FFF0246FB68D31A41F28832934201D90E
:1060F0000323E1E0734B9B6803F00C03042BEED108
:10610000B7E07B685B68022B12D10AE004F058FF0D
:106110000246FB68D31A41F28832934201D9032325
:10612000CAE0684B9B6803F00C03082BEED1A0E09B
:106130000AE004F045FF0246FB68D31A41F28832B8
:10614000934201D90323B7E05E4B9B6803F00C0335
:10615000002BEED18DE07B681B6803F00203002B5F
:1061600008D05849574B9B6823F0F0027B689B6826
:1061700013438B607B681B6803F00103002B6BD01B
:106180007B685B68012B07D14E4B1B6803F400331F
:10619000002B15D101238FE07B685B68022B07D1B0
:1061A000484B1B6803F00073002B09D1012383E0E7
:1061B000444B1B6803F00203002B01D101237BE059
:1061C0004049404B9B6823F003027B685B681343A4
:1061D0008B6004F0F5FEF8607B685B68012B12D1E0
:1061E0000AE004F0EDFE0246FB68D31A41F2883261
:1061F000934201D903235FE0324B9B6803F00C0309
:10620000042BEED128E07B685B68022B12D10AE0F8
:1062100004F0D6FE0246FB68D31A41F2883293425C
:1062200001D9032348E0274B9B6803F00C03082B9C
:10623000EED111E00AE004F0C3FE0246FB68D31A77
:1062400041F28832934201D9032335E01D4B9B680C
:1062500003F00C03002BEED1194B3A68D2B21A703E
:10626000174B1B6803F00F023B689A4201D00123D1
:1062700022E07B681B6803F00403002B08D011495F
:10628000104B9B6823F4E0527B68DB6813438B6000
:106290007B681B6803F00803002B09D00949094BF0
:1062A0009B6823F460427B681B69DB0013438B60AF
:1062B000002004F061FE002318461037BD4680BD63
:1062C000003C02400038024080B491B000AF00238F
:1062D0007B630023FB6300233B630023BB633D4BD5
:1062E0009B6803F00C03042B06D0082B07D0002B6F
:1062F00066D1394BBB6366E0384BBB6363E0354B1B
:106300005B6803F03F037B63324B5B6803F48003FD
:10631000002B1CD0314A7B6BB2FBF3F22D4B59683A
:1063200047F6C0730B4047F6C071F962F96A91FAFB
:10633000A1F1B962B96A7962796AB1FA81F1396217
:10634000396AC9B2CB4003FB02F3FB631BE0224A6C
:106350007B6BB2FBF3F21F4B596847F6C0730B40DF
:1063600047F6C071F961F96991FAA1F1B961B969AA
:1063700079617969B1FA81F139613969C9B2CB4082
:1063800003FB02F3FB63134B5B6803F440334FF4EE
:106390004032FA60FA6892FAA2F2BA60BA687A6099
:1063A0007A68B2FA82F23A603A68D2B2D3400133E4
:1063B0005B003B63FA6B3B6BB2FBF3F3BB6302E046
:1063C000054BBB6300BFBB6B18464437BD465DF849
:1063D000047B7047003802400024F40000127A0069
:1063E00080B584B000AFFFF76FFF01460F4B9B688D
:1063F00003F0F003F022FA60FA6892FAA2F2BA60AF
:10640000BA687A607A68B2FA82F23A603A68D2B2CE
:10641000D340074AD35C21FA03F3064A1360054BC5
:106420001B6818461037BD4680BD00BF00380240CB
:10643000D0B20008DC00002080B485B000AF7860E6
:106440000B46FB7013463B800023FB730023BB60AD
:106450007B681B685B6ABB60FB78002B08D17B689C
:106460001B683A8812041146BA680A439A6229E006
:106470007B681B689B6A1B0CBA681344BB600023D3
:10648000FB730DE07B681A68FB7B40339B00134471
:106490005B681B0CBA681344BB60FB7B0133FB7366
:1064A000FA7BFB78013B9A42ECDB7B681968FB784E
:1064B000013B3A8812041046BA68024340339B00FD
:1064C0000B445A60002318461437BD465DF8047B20
:1064D000704700BF80B483B000AF78600B467B800C
:1064E0007B681B687A885A62002318460C37BD46C1
:1064F0005DF8047B704700BFF0B58FB00AAF7860DD
:106500000023FB607B68002B01D10123F7E07B684F
:10651000032283F87D237868F9F7BEFE7B681B6849
:106520001846FDF767FE7B68D3F800E07E686D468D
:1065300006F110040FCC0FC50FCC0FC523682B60DC
:10654000331D0ECB7046FDF7F1FD7B681B681846C6
:106550000021FDF761FE0023FB604CE07968FA68DA
:106560001346DB009B1A9B000B44303301225A7107
:10657000FB68D8B27968FA681346DB009B1A9B0067
:106580000B44303302461A71FB6898B27968FA6896
:106590001346DB009B1A9B000B44303302465A81A2
:1065A0007968FA681346DB009B1A9B000B44303372
:1065B0000022DA717968FA681346DB009B1A9B00A7
:1065C0000B44383300225A607968FA681346DB00BE
:1065D0009B1A9B000B44383300229A607968FA6852
:1065E0001346DB009B1A9B000B44403300229A6049
:1065F000FB680133FB60FB680E2BAFD90023FB6007
:106600005AE07968FA681346DB009B1A9B000B443A
:1066100003F5EC7300225A70FB68D8B27968FA6807
:106620001346DB009B1A9B000B4403F5EC730246F8
:106630001A70FB6898B27968FA681346DB009B1AF7
:106640009B000B44303302465A817968FA6813463E
:10665000DB009B1A9B000B4403F5EC730022DA70FD
:106660007968FA681346DB009B1A9B000B4403F51C
:10667000F07300221A607968FA681346DB009B1AEF
:106680009B000B4403F5F07300225A607968FA68A6
:106690001346DB009B1A9B000B4403F5F4730022A6
:1066A0005A607B681A68FB6840339B0013440022E1
:1066B0005A60FB680133FB60FB680E2BA1D97B6835
:1066C000D3F800E07E686D4606F110040FCC0FC5CC
:1066D0000FCC0FC523682B60331D0ECB7046FDF722
:1066E000C3FD7B68012283F87D237B68002283F849
:1066F0007C237B681B681846FEF7E2FD00231846E2
:106700001437BD46F0BD00BF80B582B000AF7860E1
:106710007B6893F87C33012B01D1022312E07B6864
:10672000012283F87C237B681B681846FEF7B0FDC6
:106730007B681B681846FDF74BFD7B68002283F8D9
:106740007C23002318460837BD4680BD80B582B043
:1067500000AF78607B6893F87C33012B01D1022372
:1067600017E07B68012283F87C237B681B6818464E
:10677000FDF740FD7B681B681846FEF71FFD7B6830
:106780001B681846FEF79CFD7B68002283F87C237B
:10679000002318460837BD4680BD00BF80B58AB0CB
:1067A00000AF78607B681B68BB6100237B620023BD
:1067B0003B6200237B610023FB6100233B610023DC
:1067C000FB607B681B681846FEF71EFE0346002B25
:1067D00040F092837B681B681846FEF789FD0346EC
:1067E000002B00D188E37B681B681846FEF780FD0C
:1067F000034603F00203002B03D07B681B680222D0
:106800005A617B681B681846FEF772FD034603F465
:106810000023002B00F0B3800023FB617B681B6822
:106820001846FEF77BFD3862A5E03B6A03F00103E2
:10683000002B00F09A807B681A68FB69DBB2104677
:106840001946FEF79BFD78617B6903F00103002B7D
:106850006CD0FB695A01BB69134403F530631A46D7
:10686000012393607B681B69012B3CD17968FA692D
:106870001346DB009B1A9B000B4403F5F0731A6868
:10688000FB695901BB690B4403F530631B69C3F312
:106890001203D11A7868FA691346DB009B1A9B0031
:1068A000034403F5F87319607968FA691346DB004D
:1068B0009B1A9B000B4403F5F07359687868FA69DA
:1068C0001346DB009B1A9B00034403F5F0731B681F
:1068D00019447868FA691346DB009B1A9B0003444D
:1068E00003F5F0735960FB69DBB278681946F9F774
:1068F0001BFD7B681B69012B18D1FB69002B15D18F
:106900007968FA691346DB009B1A9B000B4403F578
:10691000F4735B68002B09D17B681A687B6803F508
:106920006073104601211A46FEF7B2FD7B6903F041
:106930000803002B0BD07868F9F7E4FCFB695A01D7
:10694000BB69134403F530631A46082393607B69DF
:1069500003F01003002B08D0FB695A01BB691344F4
:1069600003F530631A4610239360FB690133FB6122
:106970003B6A5B083B623B6A002B7FF456AF7B6847
:106980001B681846FEF7B4FC034603F48023002B73
:1069900000F0C4807B681B681846FEF7D7FC38629D
:1069A0000023FB61B6E03B6A03F00103002B00F01B
:1069B000AB807B681A68FB69DBB210461946FEF7AC
:1069C000F9FC78617B6903F00103002B5BD0FB6964
:1069D000012202FA03F33B61BB6903F50063194628
:1069E000BB6903F500635A6B3B69DB4313404B63A0
:1069F000FB695A01BB69134403F510631A4601236E
:106A000093607B681B69012B1BD17968FA69134677
:106A1000DB009B1A9B000B44383399687868FA694D
:106A20001346DB009B1A9B00034438335B68194410
:106A30007868FA691346DB009B1A9B0003443833DD
:106A40009960FB69DBB278681946F9F789FC7B68C5
:106A50001B69012B17D1FB69002B14D17968FA69E6
:106A60001346DB009B1A9B000B4440339B68002BB2
:106A700009D17B681A687B6803F5607310460121B1
:106A80001A46FEF705FD7B6903F00803002B08D0CA
:106A9000FB695A01BB69134403F510631A460823C6
:106AA00093607B6903F01003002B08D0FB695A0147
:106AB000BB69134403F510631A46102393607B6986
:106AC00003F04003002B08D0FB695A01BB69134453
:106AD00003F510631A46402393607B6903F00203B9
:106AE000002B08D0FB695A01BB69134403F51063FE
:106AF0001A46022393607B6903F08003002B03D0C6
:106B00007868F96900F076FCFB690133FB613B6A48
:106B10005B083B623B6A002B7FF445AF7B681B68D8
:106B20001846FEF7E5FB0346002B12DABB6903F5B6
:106B300000631A46BB6903F500635B6823F0010339
:106B400053607868F9F776FC7B681B684FF0004269
:106B50005A617B681B681846FEF7CAFB034603F4BC
:106B60000063002B0FD0BB6903F500639B6803F043
:106B70000103002B02D07868F9F742FC7B681B68A0
:106B80004FF400625A617B681B681846FEF7B0FB41
:106B9000034603F48053002B00F09080BB6903F59B
:106BA00000631A46BB6903F500635B6823F00103C9
:106BB00053607B681B6818460021FDF781FC0023A9
:106BC0007B6214E07B6A5A01BB69134403F51063CE
:106BD0001A46FF2393607B6A5A01BB69134403F58D
:106BE00030631A46FF2393607B6A01337B627B68C4
:106BF0005A687B6A9A42E5D8BB6903F500631A4676
:106C00004FF0FF339361BB6903F500631A46BB691C
:106C100003F50063DB6943F00113D3617B68DB6A32
:106C2000002B18D0BB6903F500631A46BB6903F556
:106C30000063D3F8843043F00B03C2F88430BB699F
:106C400003F500631A46BB6903F500635B6C43F010
:106C50000B03536415E0BB6903F500631A46BB6977
:106C600003F500635B6943F00B035361BB6903F5F4
:106C700000631A46BB6903F500631B6943F00B030D
:106C80001361BB6903F500631A46BB6903F5006332
:106C90001B6823F4FE6313607B6819687B681B69BB
:106CA000DAB27B6803F56073084611461A46FEF7B0
:106CB000EFFB7B681B684FF480525A617B681B684E
:106CC0001846FEF715FB034603F40053002B3AD099
:106CD0007B681B681846FEF7A5FB7B681B687A6813
:106CE0001268D26822F47052DA607B681B6818461A
:106CF000FDF746FC0346002B0FD17B680022DA60CB
:106D00007B684FF400725A617B681B687A6812686E
:106D1000D26842F41052DA600DE07B680322DA6038
:106D20007B6840225A617B681B687A681268D26867
:106D300042F4A052DA607868F9F73AFB7B681B6886
:106D40004FF400525A617B681B681846FEF7D0FA70
:106D5000034603F01003002B63D07B681B687A683E
:106D60001268926922F010029A61BB691B6AFB608B
:106D7000FB6803F00F021346DB009B1A9B0003F530
:106D8000EC737A681344BB60FB6803F4F0135B0C8C
:106D9000022B26D1FA6847F6F0731340002B38D047
:106DA000BB68D968FA6847F6F07313401B099BB2B9
:106DB000B8691A46FEF7F8F8BB68DA68F96847F66A
:106DC000F0730B401B091A44BB68DA60BB689A6910
:106DD000F96847F6F0730B401B091A44BB689A61C7
:106DE00017E0FB6803F4F0135B0C062B11D17B68F2
:106DF00003F56073B86919460822FEF7D5F8BB6839
:106E00009A69F96847F6F0730B401B091A44BB688E
:106E10009A617B681B687A681268926942F0100276
:106E20009A617B681B681846FEF762FA034603F016
:106E30000803002B06D07868F9F7ACFA7B681B686A
:106E400008225A617B681B681846FEF751FA034610
:106E500003F48013002B0AD0FB69DBB27868194673
:106E6000F9F714FB7B681B684FF480125A617B684A
:106E70001B681846FEF73CFA034603F40013002B88
:106E80000AD0FB69DBB278681946F9F7EDFA7B683E
:106E90001B684FF400125A617B681B681846FEF7A6
:106EA00027FA034603F08043002B07D07868F9F7F0
:106EB000FFFA7B681B684FF080425A617B681B6851
:106EC0001846FEF715FA034603F00403002B13D00F
:106ED0007B681B685B68FB60FB6803F00403002BA6
:106EE00002D07868F9F7F2FA7B681B687A68126852
:106EF0005168FA680A435A602837BD4680BD00BF12
:106F000080B582B000AF78600B46FB707B6893F869
:106F10007C33012B01D102230FE07B68012283F82F
:106F20007C237B681A68FB7810461946FEF78AF9BD
:106F30007B68002283F87C23002318460837BD466F
:106F400080BD00BF80B584B000AF786008461146B0
:106F50001A460346FB700B463B801346BB7000236A
:106F6000FB72FB785BB2002B0CDAFB7803F07F023C
:106F70001346DB009B1A9B0030337A6813440433BA
:106F8000FB600BE0FB7803F07F021346DB009B1AEB
:106F90009B0003F5EC737A681344FB60FB7803F005
:106FA0007F03DAB2FB681A70FB78DB09DBB21A46A2
:106FB000FB685A703A88FB689A60FB68BA78DA70A6
:106FC000FB685B78002B04D0FB681B789AB2FB68E7
:106FD000DA80BB78022B02D1FB6800221A717B6831
:106FE00093F87C33012B01D102230EE07B68012250
:106FF00083F87C237B681B681846F968FDF7F6FA6E
:107000007B68002283F87C23FB7A18461037BD4644
:1070100080BD00BF80B584B000AF78600B46FB70C8
:10702000FB785BB2002B0CDAFB7803F07F0213468F
:10703000DB009B1A9B0030337A6813440433FB60F7
:107040000BE0FB7803F07F021346DB009B1A9B00EA
:1070500003F5EC737A681344FB60FB7803F07F035D
:10706000DAB2FB681A70FB78DB09DBB21A46FB6800
:107070005A707B6893F87C33012B01D102230EE018
:107080007B68012283F87C237B681B681846F968BB
:10709000FDF736FB7B68002283F87C23002318462B
:1070A0001037BD4680BD00BF80B586B000AFF86028
:1070B0007A603B600B46FB72FB7A03F07F0213465B
:1070C000DB009B1A9B0003F5EC73FA6813447B61A9
:1070D0007B697A68DA607B693A685A617B69002269
:1070E0009A617B6900225A70FB7A03F07F03DAB25F
:1070F0007B691A70FB681B69012B02D17A687B6976
:107100001A61FB6893F87C33012B01D1022322E042
:10711000FB68012283F87C23FB7A03F07F03002BBA
:107120000AD1FB681A68FB681B69DBB210467969F3
:107130001A46FDF7A3FD09E0FB681A68FB681B69A6
:10714000DBB2104679691A46FDF756FBFB68002250
:1071500083F87C23002318461837BD4680BD00BF46
:1071600080B483B000AF78600B46FB70FB7803F00F
:107170007F0279681346DB009B1A9B000B4403F5E2
:10718000F8731B689BB218460C37BD465DF8047B4C
:10719000704700BF80B586B000AFF8607A603B6092
:1071A0000B46FB72FB7A03F07F021346DB009B1A4F
:1071B0009B003033FA68134404337B617B697A683F
:1071C000DA607B693A685A617B6900229A617B695F
:1071D00001225A70FB7A03F07F03DAB27B691A70DE
:1071E000FB681B69012B02D17A687B691A61FB6815
:1071F00093F87C33012B01D1022322E0FB680122AA
:1072000083F87C23FB7A03F07F03002B0AD1FB6811
:107210001A68FB681B69DBB2104679691A46FDF7EC
:107220002DFD09E0FB681A68FB681B69DBB210469C
:1072300079691A46FDF7E0FAFB68002283F87C239F
:10724000002318461837BD4680BD00BF80B584B006
:1072500000AF78600B46FB70FB785BB2002B0CDA5A
:10726000FB7803F07F021346DB009B1A9B00303350
:107270007A6813440433FB6009E0FA781346DB00B4
:107280009B1A9B0003F5EC737A681344FB60FB6860
:1072900001229A70FB7803F07F03DAB2FB681A7060
:1072A000FB78DB09DBB21A46FB685A707B6893F8FF
:1072B0007C33012B01D1022320E07B68012283F87B
:1072C0007C237B681B681846F968FDF797FEFB78FE
:1072D00003F07F03002B0CD17B6819687B681B6966
:1072E000DAB27B6803F56073084611461A46FEF76A
:1072F000CFF87B68002283F87C23002318461037E0
:10730000BD4680BD80B584B000AF78600B46FB7091
:10731000FB785BB2002B0CDAFB7803F07F0213469C
:10732000DB009B1A9B0030337A6813440433FB6004
:1073300009E0FA781346DB009B1A9B0003F5EC7317
:107340007A681344FB60FB6800229A70FB7803F0B4
:107350007F03DAB2FB681A70FB78DB09DBB21A46EE
:10736000FB685A707B6893F87C33012B01D10223B0
:107370000EE07B68012283F87C237B681B6818463B
:10738000F968FDF7ADFE7B68002283F87C230023BB
:1073900018461037BD4680BD80B582B000AF78601A
:1073A0000B46FB707B6893F87C33012B01D10223E1
:1073B0001BE07B68012283F87C23FB785BB2002B07
:1073C00009DA7B681A68FB7803F07F0310461946D8
:1073D000FDF776F804E07B681B681846FDF796F821
:1073E0007B68002283F87C23002318460837BD46BB
:1073F00080BD00BF90B58BB002AF786039607B680C
:107400001B687B610023FB6100233B613A681346E4
:10741000DB009B1A9B0030337A6813440433FB6013
:10742000FB685A69FB689B69D31AFB61FA69FB68C0
:107430009B689A4202D9FB689B68FB61FB69033336
:10744000002B00DA03339B10BB612EE0FB68D96888
:107450003B68DAB2FB699CB27B681B69DBB20093C4
:1074600078692346FDF768FDFB68DA68FB691A4412
:10747000FB68DA60FB689A69FB691A44FB689A61E9
:10748000FB685A69FB689B69D31AFB61FA69FB6860
:107490009B689A4202D9FB689B68FB61FB690333D6
:1074A000002B00DA03339B10BB613B685A017B69F8
:1074B000134403F510639B699AB2BB699A4209D3DE
:1074C000FB689A69FB685B699A4203D2FB685B6957
:1074D000002BBBD1FB69002B13DC3B68012202FAB5
:1074E00003F33B617B6903F5006319467B6903F590
:1074F00000635A6B3B69DB4313404B637868F8F7D2
:10750000F3FF002318462437BD4690BD80B487B0F2
:1075100000AF786039600023FB600023BB6000236C
:107520003B6100237B6165E17B69012202FA03F381
:10753000FB603B681A68FB681340BB60BA68FB6875
:107540009A4240F054813B685B68022B03D03B6851
:107550005B68122B22D17B69DA087B68083253F80A
:1075600022303B617B6903F007039B001A460F231F
:107570009340DB433A6913403B613B681B697A697E
:1075800002F00702920093403A6913433B617B6922
:10759000DA087B680832396943F822107B681B6877
:1075A0003B617B695B001A4603239340DB433A69E6
:1075B00013403B613B685B6803F003037A69520048
:1075C00093403A6913433B617B683A691A603B68B0
:1075D0005B68012B0BD03B685B68022B07D03B68D4
:1075E0005B68112B03D03B685B68122B2FD17B6843
:1075F0009B683B617B695B001A4603239340DB4336
:107600003A6913403B613B68DB687A6952009340FA
:107610003A6913433B617B683A699A607B685B68AF
:107620003B617B69012202FA03F3DB433A691340B1
:107630003B613B685B6803F010031A097B6902FA3F
:1076400003F33A6913433B617B683A695A607B688C
:10765000DB683B617B695B001A4603239340DB4395
:107660003A6913403B613B689B687A6952009340DA
:107670003A6913433B617B683A69DA603B685B684F
:1076800003F08053002B00F0B2805F4A5E4B5B6CCE
:1076900043F4804353645D4A7B699B08023352F88C
:1076A00023303B617B6903F003039B001A460F23E1
:1076B0009340DB433A6913403B617B68544A9342F1
:1076C00031D07B68534A93422BD07B68524A934215
:1076D00025D07B68514A93421FD07B68504A934221
:1076E00019D07B684F4A934213D07B684E4A93422D
:1076F0000DD07B684D4A934207D07B684C4A934239
:1077000001D1082310E009230EE007230CE0062333
:107710000AE0052308E0042306E0032304E0022333
:1077200002E0012300E000237A6902F003029200E4
:1077300093403A6913433B6134497B699B080233A8
:107740003A6941F823203B4B1B683B61BB68DB4334
:107750003A6913403B613B685B6803F48033002B5C
:1077600003D03A69BB6813433B61324A3B691360FB
:10777000304B5B683B61BB68DB433A6913403B615C
:107780003B685B6803F40033002B03D03A69BB68A5
:1077900013433B61274A3B695360264B9B683B611F
:1077A000BB68DB433A6913403B613B685B6803F4A9
:1077B0008013002B03D03A69BB6813433B611D4A19
:1077C0003B6993601B4BDB683B61BB68DB433A69F9
:1077D00013403B613B685B6803F40013002B03D04C
:1077E0003A69BB6813433B61124A3B69D3607B69CA
:1077F00001337B617B690F2B7FF696AE1C37BD464C
:107800005DF8047B704700BF00380240003801403B
:10781000000002400004024000080240000C024048
:10782000001002400014024000180240001C0240F8
:1078300000200240003C014080B485B000AF786079
:107840000023FB607B68002B01D101235BE07B6898
:10785000022283F835207B681B681B68FB60FA688E
:107860002C4B1340FB607B685A687B689B681A430B
:107870007B68DB681A437B681B691A437B685B691A
:107880001A437B689B691A437B68DB691A437B68F0
:107890001B6A1343FA681343FB607B685B6A042B23
:1078A00007D17B68DA6A7B681B6B1343FA68134362
:1078B000FB607B681B68FA681A607B681B685B6901
:1078C000FB60FB6823F00703FB607B685B6AFA6878
:1078D0001343FB607B685B6A042B04D17B689B6A63
:1078E000FA681343FB607B681B68FA685A617B681F
:1078F0000022DA647B68012283F835207B6800224D
:1079000083F83420002318461437BD465DF8047B05
:10791000704700BF3F8010F080B584B000AFF860C2
:10792000B9607A603B60FB6893F83430012B01D179
:10793000022346E0FB68012283F83420FB68022220
:1079400083F83520FB681B68FA681268126822F019
:1079500001021A60F868B9687A683B6803F09AF91E
:10796000FB681B68FA681268126842F010021A601D
:10797000FB681B68FA681268126842F008021A6015
:10798000FB681B68FA681268126842F004021A6009
:10799000FB681B68FA681268526942F080025A61FB
:1079A000FB681B68FA681268126842F002021A60EB
:1079B000FB681B68FA681268126842F001021A60DC
:1079C000002318461037BD4680BD00BF80B582B089
:1079D00000AF78607B681B681A46784B9A4272D970
:1079E000774B5A687B681B681946764B994262D080
:1079F0007B681B681946744B99425AD07B681B6898
:107A00001946724B994252D07B681B681946704BDD
:107A100099424AD07B681B6819466E4B994241D007
:107A20007B681B6819466C4B994238D07B681B6891
:107A300019466A4B99422FD07B681B681946684BE0
:107A4000994226D07B681B681946664B99421DD027
:107A50007B681B681946644B994214D07B681B688D
:107A60001946624B99420BD07B681B681946604BE4
:107A7000994202D14FF400231EE04FF000731BE047
:107A80004FF4002318E04FF4002315E04FF40023D7
:107A900012E04FF400730FE04FF400730CE04FF46A
:107AA000007309E04FF4007306E0082304E00823A4
:107AB00002E0082300E008231340002B14BF012339
:107AC0000023DBB29FE17B681B681A46494B9A4250
:107AD00040F292803A4B1A687B681B681946394B12
:107AE000994262D07B681B681946374B99425AD03D
:107AF0007B681B681946354B994252D07B681B68DE
:107B00001946334B99424AD07B681B681946314B62
:107B1000994241D07B681B6819462F4B994238D057
:107B20007B681B6819462D4B99422FD07B681B68D8
:107B300019462B4B994226D07B681B681946294B66
:107B400099421DD07B681B681946274B994214D077
:107B50007B681B681946254B99420BD07B681B68D4
:107B60001946234B994202D14FF400231EE04FF0F7
:107B700000731BE04FF4002318E04FF4002315E0DE
:107B80004FF4002312E04FF400730FE04FF4007342
:107B90000CE04FF4007309E04FF4007306E0082393
:107BA00004E0082302E0082300E008231340002B30
:107BB00014BF01230023DBB225E100BF586402405B
:107BC0000064024010600240106402407060024095
:107BD00070640240286002402864024088600240CD
:107BE000886402404060024040640240A06002405D
:107BF000A0640240B86002407B681B681A46704B64
:107C00009A4272D96F4B5A687B681B6819466E4B53
:107C1000994262D07B681B6819466C4B99425AD0D6
:107C20007B681B6819466A4B994252D07B681B6877
:107C30001946684B99424AD07B681B681946664BC7
:107C4000994241D07B681B681946644B994238D0F1
:107C50007B681B681946624B99422FD07B681B6872
:107C60001946604B994226D07B681B6819465E4BCB
:107C700099421DD07B681B6819465C4B994214D011
:107C80007B681B6819465A4B99420BD07B681B686E
:107C90001946584B994202D14FF400231EE04FF091
:107CA00000731BE04FF4002318E04FF4002315E0AD
:107CB0004FF4002312E04FF400730FE04FF4007311
:107CC0000CE04FF4007309E04FF4007306E0082362
:107CD00004E0082302E0082300E008231340002BFF
:107CE00014BF01230023DBB28DE0364B1A687B689A
:107CF0001B681946344B99427ED07B681B68194635
:107D0000324B99425AD07B681B681946304B9942D6
:107D100052D07B681B6819462E4B99424AD07B682B
:107D20001B6819462C4B994241D07B681B68194649
:107D30002A4B994238D07B681B681946284B9942D8
:107D40002FD07B681B681946264B994226D07B684A
:107D50001B681946244B99421DD07B681B68194645
:107D6000224B994214D07B681B681946204B9942DC
:107D70000BD07B681B6819461E4B994202D14FF409
:107D800000233AE04FF0007337E04FF4002334E073
:107D90004FF4002331E04FF400232EE04FF4007342
:107DA0002BE04FF4007328E04FF4007325E04FF40C
:107DB000007322E0082320E008231EE008231CE0D3
:107DC00058600240006002401060024010640240AF
:107DD00070600240706402402860024028640240E3
:107DE0008860024088640240406002404064024073
:107DF000A0600240A064024008231340002B14BF7F
:107E000001230023DBB2002B00F010827B681B688B
:107E10001B6803F00403002B00F008827B681B68DA
:107E20007A681268126822F004021A607B681B6884
:107E30001A46A04B9A426CD99F4A7B681B68194628
:107E40009E4B994262D07B681B6819469C4B9942B5
:107E50005AD07B681B6819469A4B994252D07B686E
:107E60001B681946984B99424AD07B681B68194693
:107E7000964B994241D07B681B681946944B9942B6
:107E800038D07B681B681946924B99422FD07B688B
:107E90001B681946904B994226D07B681B6819468F
:107EA0008E4B99421DD07B681B6819468C4B9942BA
:107EB00014D07B681B6819468A4B99420BD07B68AB
:107EC0001B681946884B994202D14FF400231EE0EB
:107ED0004FF000731BE04FF4002318E04FF4002331
:107EE00015E04FF4002312E04FF400730FE04FF45D
:107EF00000730CE04FF4007309E04FF4007306E0E8
:107F0000082304E0082302E0082300E00823D360EC
:107F100076E17B681B681A46744B9A426CD9664AB4
:107F20007B681B681946654B994262D07B681B6869
:107F30001946634B99425AD07B681B681946614BBE
:107F4000994252D07B681B6819465F4B99424AD0D0
:107F50007B681B6819465D4B994241D07B681B6862
:107F600019465B4B994238D07B681B681946594BC0
:107F700099422FD07B681B681946574B994226D0EF
:107F80007B681B681946554B99421DD07B681B685E
:107F90001946534B994214D07B681B681946514BC4
:107FA00099420BD07B681B6819464F4B994202D10E
:107FB0004FF400231EE04FF000731BE04FF400234A
:107FC00018E04FF4002315E04FF4002312E04FF4C3
:107FD00000730FE04FF400730CE04FF4007309E0FE
:107FE0004FF4007306E0082304E0082302E00823AE
:107FF00000E00823936003E17B681B681A463C4B52
:108000009A4240F291803B4A7B681B6819462B4B91
:10801000994200F086807B681B681946284B99427C
:108020007DD07B681B681946264B994275D07B68CA
:108030001B681946244B99426DD07B681B68194612
:10804000224B994264D07B681B681946204B9942A9
:108050005BD07B681B6819461E4B994252D07B68E7
:108060001B6819461C4B994249D07B681B6819460E
:108070001A4B994240D07B681B681946184B9942AD
:1080800014D07B681B681946164B99420BD07B684D
:108090001B681946144B994202D14FF4002341E06A
:1080A0004FF000733EE04FF400233BE04FF4002319
:1080B00038E000BF58640240006402401060024093
:1080C0001064024070600240706402402860024008
:1080D0002864024088600240886402404060024098
:1080E00040640240A0600240A0640240B8600240C8
:1080F00058600240006002404FF4002312E04FF449
:1081000000730FE04FF400730CE04FF4007309E0CC
:108110004FF4007306E0082304E0082302E008237C
:1081200000E00823D3606BE07B4A7B681B6819463C
:108130007A4B994262D07B681B681946784B99420A
:108140005AD07B681B681946764B994252D07B689F
:108150001B681946744B99424AD07B681B681946C4
:10816000724B994241D07B681B681946704B99420B
:1081700038D07B681B6819466E4B99422FD07B68BC
:108180001B6819466C4B994226D07B681B681946C0
:108190006A4B99421DD07B681B681946684B99420F
:1081A00014D07B681B681946664B99420BD07B68DC
:1081B0001B681946644B994202D14FF400231EE01C
:1081C0004FF000731BE04FF4002318E04FF400233E
:1081D00015E04FF4002312E04FF400730FE04FF46A
:1081E00000730CE04FF4007309E04FF4007306E0F5
:1081F000082304E0082302E0082300E0082393603A
:108200007B68DB6C43F001027B68DA647B680422E4
:1082100083F835207B68002283F834207B689B6CD0
:10822000002B03D07B689B6C786898477B681B6841
:108230001A46464B9A4240F28F80454B5A687B68FB
:108240001B681946354B99425ED07B681B681946FE
:10825000334B994256D07B681B681946314B994283
:108260004ED07B681B6819462F4B994246D07B68DD
:108270001B6819462D4B99423ED07B681B681946F6
:108280002B4B994236D07B681B681946294B994283
:108290002ED07B681B681946274B994226D07B68F5
:1082A0001B681946254B99421DD07B681B681946EF
:1082B000234B994214D07B681B681946214B994285
:1082C0000BD07B681B6819461F4B994202D14FF4B3
:1082D00080331AE04FF4800317E04FF4803314E04A
:1082E0004FF4803311E04FF480330EE040230CE074
:1082F00040230AE0402308E0402306E0154B04E059
:10830000144B02E0134B00E0124B1340002B14BF40
:1083100001230023DBB29AE10060024010600240BA
:1083200010640240706002407064024028600240A5
:108330002864024088600240886402404060024035
:1083400040640240A0600240A064024058640240C1
:1083500000640240010080007B681B681A469A4B4B
:108360009A426ED9994B1A687B681B681946984BDC
:1083700099425ED07B681B681946964B994256D04D
:108380007B681B681946944B99424ED07B681B68EA
:108390001946924B994246D07B681B681946904B10
:1083A00099423ED07B681B6819468E4B994236D065
:1083B0007B681B6819468C4B99422ED07B681B68E2
:1083C00019468A4B994226D07B681B681946884B10
:1083D00099421DD07B681B681946864B994214D080
:1083E0007B681B681946844B99420BD07B681B68DD
:1083F0001946824B994202D14FF480331AE04FF470
:10840000800317E04FF4803314E04FF4803311E021
:108410004FF480330EE040230CE040230AE0402379
:1084200008E0402306E0764B04E0754B02E0744B15
:1084300000E0734B1340002B14BF01230023DBB279
:1084400005E17B681B681A466E4B9A426ED96E4BEB
:108450005A687B681B6819465D4B99425ED07B6801
:108460001B6819465B4B994256D07B681B681946BE
:10847000594B99424ED07B681B681946574B99421D
:1084800046D07B681B681946554B99423ED07B68A5
:108490001B681946534B994236D07B681B681946B6
:1084A000514B99422ED07B681B6819464F4B99421D
:1084B00026D07B681B6819464D4B99421DD07B68BE
:1084C0001B6819464B4B994214D07B681B681946B0
:1084D000494B99420BD07B681B681946474B994220
:1084E00002D14FF480331AE04FF4800317E04FF4C9
:1084F000803314E04FF4803311E04FF480330EE00A
:1085000040230CE040230AE0402308E0402306E03B
:108510003B4B04E03A4B02E0394B00E0384B134050
:10852000002B14BF01230023DBB290E0364B1A6806
:108530007B681B681946264B994200F081807B6856
:108540001B681946234B994278D07B681B681946F3
:10855000214B994270D07B681B6819461F4B99428A
:1085600068D07B681B6819461D4B994260D07B68B8
:108570001B6819461B4B994258D07B681B681946EB
:10858000194B994250D07B681B681946174B99428A
:1085900048D07B681B681946154B99423FD07B68D1
:1085A0001B681946134B994236D07B681B681946E5
:1085B000114B99422DD07B681B6819460F4B99428D
:1085C00024D14FF480333CE0B860024000640240A4
:1085D000106002401064024070600240706402400B
:1085E000286002402864024088600240886402409B
:1085F0004060024040640240A0600240A06402402B
:108600000100800058600240006002404FF4800387
:1086100017E04FF4803314E04FF4803311E04FF44F
:1086200080330EE040230CE040230AE0402308E0C2
:10863000402306E07F4B04E07E4B02E07D4B00E0F0
:108640007C4B1340002B14BF01230023DBB2002B13
:1086500000F01C827B681B685B6903F08003002BC1
:1086600000F014827B681B687A681268526922F0F5
:1086700080025A617B681B681A466F4B9A4268D920
:108680006E4A7B681B6819466D4B99425ED07B68C9
:108690001B6819466B4B994256D07B681B6819467C
:1086A000694B99424ED07B681B681946674B9942CB
:1086B00046D07B681B681946654B99423ED07B6863
:1086C0001B681946634B994236D07B681B68194674
:1086D000614B99422ED07B681B6819465F4B9942CB
:1086E00026D07B681B6819465D4B99421DD07B687C
:1086F0001B6819465B4B994214D07B681B6819466E
:10870000594B99420BD07B681B681946574B9942CD
:1087100002D14FF480331AE04FF4800317E04FF496
:10872000803314E04FF4803311E04FF480330EE0D7
:1087300040230CE040230AE0402308E0402306E009
:108740003C4B04E03B4B02E03A4B00E0394BD3603A
:1087500086E17B681B681A46454B9A4240F28A8044
:10876000364A7B681B681946354B99425ED07B6858
:108770001B681946334B994256D07B681B681946D3
:10878000314B99424ED07B681B6819462F4B99425A
:1087900046D07B681B6819462D4B99423ED07B68BA
:1087A0001B6819462B4B994236D07B681B681946CB
:1087B000294B99422ED07B681B681946274B99425A
:1087C00026D07B681B681946254B99421DD07B68D3
:1087D0001B681946234B994214D07B681B681946C5
:1087E000214B99420BD07B681B6819461F4B99425D
:1087F00002D14FF480331AE04FF4800317E04FF4B6
:10880000803314E04FF4803311E04FF480330EE0F6
:1088100040230CE040230AE0402308E0402306E028
:10882000044B04E0034B02E0024B00E0014B936079
:1088300016E100BF0100800058640240006402405D
:108840001060024010640240706002407064024098
:108850002860024028640240886002408864024028
:108860004060024040640240A0600240A0640240B8
:10887000B86002407B681B681A46694B9A4268D907
:10888000684A7B681B681946674B99425ED07B68D3
:108890001B681946654B994256D07B681B68194680
:1088A000634B99424ED07B681B681946614B9942D5
:1088B00046D07B681B6819465F4B99423ED07B6867
:1088C0001B6819465D4B994236D07B681B68194678
:1088D0005B4B99422ED07B681B681946594B9942D5
:1088E00026D07B681B681946574B99421DD07B6880
:1088F0001B681946554B994214D07B681B68194672
:10890000534B99420BD07B681B681946514B9942D7
:1089100002D14FF480331AE04FF4800317E04FF494
:10892000803314E04FF4803311E04FF480330EE0D5
:1089300040230CE040230AE0402308E0402306E007
:10894000454B04E0444B02E0434B00E0424BD36014
:1089500086E0344A7B681B681946334B99427DD0C8
:108960007B681B681946314B994256D07B681B685F
:1089700019462F4B99424ED07B681B6819462D4BE8
:10898000994246D07B681B6819462B4B99423ED0D2
:108990007B681B681946294B994236D07B681B6857
:1089A0001946274B99422ED07B681B681946254BE8
:1089B000994226D07B681B681946234B99421DD0EB
:1089C0007B681B681946214B994214D07B681B6851
:1089D00019461F4B99420BD07B681B6819461D4BEB
:1089E000994202D14FF4803339E04FF4800336E0EE
:1089F0004FF4803333E04FF4803330E04FF4803372
:108A00002DE040232BE0402329E0402327E04023B2
:108A100025E0114B23E0104B21E00F4B1FE000BF7E
:108A20005860024000600240106002401064024042
:108A30007060024070640240286002402864024076
:108A40008860024088640240406002404064024006
:108A5000A0600240A064024001008000854B93604A
:108A60007B68DB6C43F002027B68DA647B6804227B
:108A700083F835207B68002283F834207B689B6C68
:108A8000002B03D07B689B6C786898477B681B68D9
:108A90001A46794B9A4272D9784B5A687B681B68A0
:108AA0001946774B994262D07B681B681946754B13
:108AB00099425AD07B681B681946734B994252D031
:108AC0007B681B681946714B99424AD07B681B68CA
:108AD00019466F4B994241D07B681B6819466D4B14
:108AE000994238D07B681B6819466B4B99422FD04E
:108AF0007B681B681946694B994226D07B681B68C6
:108B00001946674B99421DD07B681B681946654B17
:108B1000994214D07B681B681946634B99420BD06D
:108B20007B681B681946614B994202D14FF4802340
:108B30001EE04FF080731BE04FF4802318E04FF4E9
:108B4000802315E04FF4802312E04FF480730FE090
:108B50004FF480730CE04FF4807309E04FF480739E
:108B600006E0534B04E0524B02E0514B00E0504B07
:108B70001340002B14BF01230023DBB2A7E17B6865
:108B80001B681A464B4B9A4240F296803B4B1A6840
:108B90007B681B6819463A4B994262D07B681B6818
:108BA0001946384B99425AD07B681B681946364B98
:108BB000994252D07B681B681946344B99424AD07F
:108BC0007B681B681946324B994241D07B681B6811
:108BD0001946304B994238D07B681B6819462E4B9A
:108BE00099422FD07B681B6819462C4B994226D09E
:108BF0007B681B6819462A4B99421DD07B681B680D
:108C00001946284B994214D07B681B681946264B9D
:108C100099420BD07B681B681946244B994202D1BC
:108C20004FF480231EE04FF080731BE04FF480234D
:108C300018E04FF4802315E04FF4802312E04FF446
:108C400080730FE04FF480730CE04FF4807309E001
:108C50004FF4807306E0164B04E0154B02E0144B12
:108C600000E0134B1340002B14BF01230023DBB2A1
:108C70002DE100BF01008000586402400064024002
:108C80001060024010640240706002407064024054
:108C900028600240286402408860024088640240E4
:108CA0004060024040640240A0600240A064024074
:108CB00004008000B86002407B681B681A46714B54
:108CC0009A4272D9704B5A687B681B6819466F4B81
:108CD000994262D07B681B6819466D4B99425AD005
:108CE0007B681B6819466B4B994252D07B681B68A6
:108CF0001946694B99424AD07B681B681946674BF5
:108D0000994241D07B681B681946654B994238D01F
:108D10007B681B681946634B99422FD07B681B68A0
:108D20001946614B994226D07B681B6819465F4BF8
:108D300099421DD07B681B6819465D4B994214D03F
:108D40007B681B6819465B4B99420BD07B681B689C
:108D50001946594B994202D14FF480231EE04FF03F
:108D600080731BE04FF4802318E04FF4802315E05C
:108D70004FF4802312E04FF480730FE04FF48073C0
:108D80000CE04FF4807309E04FF4807306E04B4B26
:108D900004E04A4B02E0494B00E0484B1340002BF3
:108DA00014BF01230023DBB291E0374B1A687B68C4
:108DB0001B681946354B994200F082807B681B681E
:108DC0001946334B99425AD07B681B681946314B80
:108DD000994252D07B681B6819462F4B99424AD062
:108DE0007B681B6819462D4B994241D07B681B68F4
:108DF00019462B4B994238D07B681B681946294B82
:108E000099422FD07B681B681946274B994226D080
:108E10007B681B681946254B99421DD07B681B68EF
:108E20001946234B994214D07B681B681946214B85
:108E300099420BD07B681B6819461F4B994202D19F
:108E40004FF480233DE04FF080733AE04FF48023ED
:108E500037E04FF4802334E04FF4802331E04FF4C7
:108E600080732EE04FF480732BE04FF4807328E082
:108E70004FF4807325E0114B23E0104B21E00F4BA2
:108E80001FE000BF586002400060024010600240D6
:108E9000106402407060024070640240286002402A
:108EA00028640240886002408864024040600240BA
:108EB00040640240A0600240A064024004008000C0
:108EC000804B1340002B14BF01230023DBB2002B87
:108ED00000F02C827B681B681B6803F00203002BE8
:108EE00000F024827B681B687A681268126822F09E
:108EF00002021A607B681B681A46734B9A426CD94F
:108F0000724A7B681B681946714B994262D07B6834
:108F10001B6819466F4B99425AD07B681B681946EB
:108F20006D4B994252D07B681B6819466B4B994236
:108F30004AD07B681B681946694B994241D07B68CF
:108F40001B681946674B994238D07B681B681946E5
:108F5000654B99422FD07B681B681946634B994239
:108F600026D07B681B681946614B99421DD07B68EF
:108F70001B6819465F4B994214D07B681B681946E1
:108F80005D4B99420BD07B681B6819465B4B99423D
:108F900002D14FF480231EE04FF080731BE04FF4AA
:108FA000802318E04FF4802315E04FF4802312E073
:108FB0004FF480730FE04FF480730CE04FF4807334
:108FC00009E04FF4807306E03E4B04E03D4B02E0C5
:108FD0003C4B00E03B4BD36092E17B681B681A4638
:108FE000474B9A4240F28E80384A7B681B6819468C
:108FF000374B994262D07B681B681946354B9942C2
:109000005AD07B681B681946334B994252D07B6813
:109010001B681946314B99424AD07B681B68194638
:109020002F4B994241D07B681B6819462D4B9942C2
:1090300038D07B681B6819462B4B99422FD07B6830
:109040001B681946294B994226D07B681B68194634
:10905000274B99421DD07B681B681946254B9942C6
:1090600014D07B681B681946234B99420BD07B6850
:109070001B681946214B994202D14FF480231EE010
:109080004FF080731BE04FF4802318E04FF48023EF
:1090900015E04FF4802312E04FF480730FE04FF49B
:1090A00080730CE04FF4807309E04FF4807306E0A6
:1090B000044B04E0034B02E0024B00E0014B9360E1
:1090C0001EE100BF040080005864024000640240BA
:1090D0001060024010640240706002407064024000
:1090E0002860024028640240886002408864024090
:1090F0004060024040640240A0600240A064024020
:10910000B86002407B681B681A466D4B9A426CD966
:109110006C4A7B681B6819466B4B994262D07B682E
:109120001B681946694B99425AD07B681B681946DF
:10913000674B994252D07B681B681946654B994230
:109140004AD07B681B681946634B994241D07B68C3
:109150001B681946614B994238D07B681B681946D9
:109160005F4B99422FD07B681B6819465D4B994233
:1091700026D07B681B6819465B4B99421DD07B68E3
:109180001B681946594B994214D07B681B681946D5
:10919000574B99420BD07B681B681946554B994237
:1091A00002D14FF480231EE04FF080731BE04FF498
:1091B000802318E04FF4802315E04FF4802312E061
:1091C0004FF480730FE04FF480730CE04FF4807322
:1091D00009E04FF4807306E0474B04E0464B02E0A1
:1091E000454B00E0444BD3608AE0364A7B681B68FD
:1091F0001946354B994200F081807B681B681946FF
:10920000324B99425AD07B681B681946304B9942C1
:1092100052D07B681B6819462E4B99424AD07B6816
:109220001B6819462C4B994241D07B681B68194634
:109230002A4B994238D07B681B681946284B9942C3
:109240002FD07B681B681946264B994226D07B6835
:109250001B681946244B99421DD07B681B68194630
:10926000224B994214D07B681B681946204B9942C7
:109270000BD07B681B6819461E4B994202D14FF4F4
:1092800080233CE04FF0807339E04FF4802336E0D8
:109290004FF4802333E04FF4802330E04FF48073A9
:1092A0002DE04FF480732AE04FF4807327E04FF4F1
:1092B000807324E0104B22E00F4B20E00E4B1EE0A9
:1092C000586002400060024010600240106402409A
:1092D00070600240706402402860024028640240CE
:1092E000886002408864024040600240406402405E
:1092F000A0600240A064024004008000854B93609F
:109300007B68DB6C43F004027B68DA647B680422D0
:1093100083F835207B68002283F834207B689B6CBF
:10932000002B03D07B689B6C786898477B681B6830
:109330001A46794B9A4272D9784B5A687B681B68F7
:109340001946774B994262D07B681B681946754B6A
:1093500099425AD07B681B681946734B994252D088
:109360007B681B681946714B99424AD07B681B6821
:1093700019466F4B994241D07B681B6819466D4B6B
:10938000994238D07B681B6819466B4B99422FD0A5
:109390007B681B681946694B994226D07B681B681D
:1093A0001946674B99421DD07B681B681946654B6F
:1093B000994214D07B681B681946634B99420BD0C5
:1093C0007B681B681946614B994202D14FF48013A8
:1093D0001EE04FF080631BE04FF4801318E04FF461
:1093E000801315E04FF4801312E04FF480630FE018
:1093F0004FF480630CE04FF4806309E04FF4806326
:1094000006E0102304E0102302E0102300E0102304
:109410001340002B14BF01230023DBB2A1E17B68C2
:109420001B681A464A4B9A4240F294803B4B1A689A
:109430007B681B6819463A4B994262D07B681B686F
:109440001946384B99425AD07B681B681946364BEF
:10945000994252D07B681B681946344B99424AD0D6
:109460007B681B681946324B994241D07B681B6868
:109470001946304B994238D07B681B6819462E4BF1
:1094800099422FD07B681B6819462C4B994226D0F5
:109490007B681B6819462A4B99421DD07B681B6864
:1094A0001946284B994214D07B681B681946264BF5
:1094B00099420BD07B681B681946244B994202D114
:1094C0004FF480131EE04FF080631BE04FF48013D5
:1094D00018E04FF4801315E04FF4801312E04FF4BE
:1094E00080630FE04FF480630CE04FF4806309E089
:1094F0004FF4806306E0102304E0102302E0102301
:1095000000E010231340002B14BF01230023DBB223
:1095100027E100BF0400800058640240006402405C
:1095200010600240106402407060024070640240AB
:10953000286002402864024088600240886402403B
:109540004060024040640240A0600240A0640240CB
:10955000B86002407B681B681A46704B9A4272D909
:109560006F4B5A687B681B6819466E4B994262D0F4
:109570007B681B6819466C4B99425AD07B681B6804
:1095800019466A4B994252D07B681B681946684B52
:1095900099424AD07B681B681946664B994241D074
:1095A0007B681B681946644B994238D07B681B68FE
:1095B0001946624B99422FD07B681B681946604B55
:1095C000994226D07B681B6819465E4B99421DD094
:1095D0007B681B6819465C4B994214D07B681B68FA
:1095E00019465A4B99420BD07B681B681946584B59
:1095F000994202D14FF480131EE04FF080631BE0CC
:109600004FF4801318E04FF4801315E04FF48013EB
:1096100012E04FF480630FE04FF480630CE04FF4EE
:10962000806309E04FF4806306E0102304E0102318
:1096300002E0102300E010231340002B14BF01238D
:109640000023DBB28DE0364B1A687B681B68194635
:10965000344B99427ED07B681B681946324B994245
:109660005AD07B681B681946304B994252D07B68B0
:109670001B6819462E4B99424AD07B681B681946D5
:109680002C4B994241D07B681B6819462A4B994262
:1096900038D07B681B681946284B99422FD07B68CD
:1096A0001B681946264B994226D07B681B681946D1
:1096B000244B99421DD07B681B681946224B994266
:1096C00014D07B681B681946204B99420BD07B68ED
:1096D0001B6819461E4B994202D14FF480133AE0A1
:1096E0004FF0806337E04FF4801334E04FF4801381
:1096F00031E04FF480132EE04FF480632BE04FF401
:10970000806328E04FF4806325E04FF4806322E01B
:10971000102320E010231EE010231CE058600240BC
:10972000006002401060024010640240706002401D
:109730007064024028600240286402408860024051
:10974000886402404060024040640240A0600240E1
:10975000A064024010231340002B14BF01230023F8
:10976000DBB2002B00F033847B681B681B6803F0BE
:109770000803002B00F02B847B681B681B6803F434
:109780008023002B00F003827B681B681A46A04BE5
:109790009A426CD99F4A7B681B6819469E4B994236
:1097A00062D07B681B6819469C4B99425AD07B68F3
:1097B0001B6819469A4B994252D07B681B68194620
:1097C000984B99424AD07B681B681946964B994240
:1097D00041D07B681B681946944B994238D07B680E
:1097E0001B681946924B99422FD07B681B6819461B
:1097F000904B994226D07B681B6819468E4B994244
:109800001DD07B681B6819468C4B994214D07B682D
:109810001B6819468A4B99420BD07B681B68194616
:10982000884B994202D14FF480131EE04FF08063C1
:109830001BE04FF4801318E04FF4801315E04FF451
:10984000801312E04FF480630FE04FF480630CE06C
:109850004FF4806309E04FF4806306E0102304E0D6
:10986000102302E0102300E01023D36076E17B6830
:109870001B681A46744B9A426CD9664A7B681B680F
:109880001946654B994262D07B681B681946634B49
:1098900099425AD07B681B681946614B994252D055
:1098A0007B681B6819465F4B99424AD07B681B68EE
:1098B00019465D4B994241D07B681B6819465B4B4A
:1098C000994238D07B681B681946594B99422FD072
:1098D0007B681B681946574B994226D07B681B68EA
:1098E0001946554B99421DD07B681B681946534B4E
:1098F000994214D07B681B681946514B99420BD092
:109900007B681B6819464F4B994202D14FF4801374
:109910001EE04FF080631BE04FF4801318E04FF41B
:10992000801315E04FF4801312E04FF480630FE0D2
:109930004FF480630CE04FF4806309E04FF48063E0
:1099400006E0102304E0102302E0102300E01023BF
:10995000936003E17B681B681A463C4B9A4240F2D5
:1099600091803B4A7B681B6819462B4B994200F05B
:1099700086807B681B681946284B99427DD07B689E
:109980001B681946264B994275D07B681B6819469F
:10999000244B99426DD07B681B681946224B994233
:1099A00064D07B681B681946204B99425BD07B686A
:1099B0001B6819461E4B994252D07B681B6819469A
:1099C0001C4B994249D07B681B6819461A4B994237
:1099D00040D07B681B681946184B994214D07B68AD
:1099E0001B681946164B99420BD07B681B681946B9
:1099F000144B994202D14FF4801341E04FF0806341
:109A00003EE04FF480133BE04FF4801338E000BF9A
:109A1000586402400064024010600240106402403A
:109A20007060024070640240286002402864024076
:109A30008860024088640240406002404064024006
:109A4000A0600240A0640240B8600240586002403A
:109A5000006002404FF4801312E04FF480630FE087
:109A60004FF480630CE04FF4806309E04FF48063AF
:109A700006E0102304E0102302E0102300E010238E
:109A8000D3606BE0834A7B681B681946824B99421E
:109A900062D07B681B681946804B99425AD07B681C
:109AA0001B6819467E4B994252D07B681B68194649
:109AB0007C4B99424AD07B681B6819467A4B994285
:109AC00041D07B681B681946784B994238D07B6837
:109AD0001B681946764B99422FD07B681B68194644
:109AE000744B994226D07B681B681946724B994289
:109AF0001DD07B681B681946704B994214D07B6857
:109B00001B6819466E4B99420BD07B681B6819463F
:109B10006C4B994202D14FF480131EE04FF08063EA
:109B20001BE04FF4801318E04FF4801315E04FF45E
:109B3000801312E04FF480630FE04FF480630CE079
:109B40004FF4806309E04FF4806306E0102304E0E3
:109B5000102302E0102300E0102393607B681B6851
:109B60001B6803F40023002B04D17B68312283F8A7
:109B7000352024E27B681B681B6803F40023002B5C
:109B800000F01D827B68412283F8352017E27B6854
:109B90001B681B6803F48073002B07D17B681B686C
:109BA0007A681268126822F008021A607B681B68E3
:109BB0001A46454B9A4240F28B80444A7B681B68A8
:109BC0001946354B994262D07B681B681946334B66
:109BD00099425AD07B681B681946314B994252D042
:109BE0007B681B6819462F4B99424AD07B681B68DB
:109BF00019462D4B994241D07B681B6819462B4B67
:109C0000994238D07B681B681946294B99422FD05E
:109C10007B681B681946274B994226D07B681B68D6
:109C20001946254B99421DD07B681B681946234B6A
:109C3000994214D07B681B681946214B99420BD07E
:109C40007B681B6819461F4B994202D14FF4801361
:109C50001EE04FF080631BE04FF4801318E04FF4D8
:109C6000801315E04FF4801312E04FF480630FE08F
:109C70004FF480630CE04FF4806309E04FF480639D
:109C800006E0102304E0102302E0102300E010237C
:109C9000D36090E100600240106002401064024016
:109CA00070600240706402402860024028640240F4
:109CB0008860024088640240406002404064024084
:109CC000A0600240A0640240586402400064024068
:109CD0007B681B681A469F4B9A426CD99E4A7B68E8
:109CE0001B6819469D4B994262D07B681B681946D8
:109CF0009B4B99425AD07B681B681946994B9942F5
:109D000052D07B681B681946974B99424AD07B68B2
:109D10001B681946954B994241D07B681B681946D0
:109D2000934B994238D07B681B681946914B9942F6
:109D30002FD07B681B6819468F4B994226D07B68D1
:109D40001B6819468D4B99421DD07B681B681946CC
:109D50008B4B994214D07B681B681946894B9942FA
:109D60000BD07B681B681946874B994202D14FF490
:109D700080131EE04FF080631BE04FF4801318E067
:109D80004FF4801315E04FF4801312E04FF480631A
:109D90000FE04FF480630CE04FF4806309E04FF470
:109DA000806306E0102304E0102302E0102300E0AB
:109DB00010239360FFE07B681B681A46734B9A423E
:109DC0006CD9734A7B681B681946644B994262D010
:109DD0007B681B681946624B99425AD07B681B68A6
:109DE0001946604B994252D07B681B6819465E4BFE
:109DF00099424AD07B681B6819465C4B994241D016
:109E00007B681B6819465A4B994238D07B681B689F
:109E10001946584B99422FD07B681B681946564B00
:109E2000994226D07B681B681946544B99421DD035
:109E30007B681B681946524B994214D07B681B689B
:109E40001946504B99420BD07B681B6819464E4B04
:109E5000994202D14FF480131EE04FF080631BE063
:109E60004FF4801318E04FF4801315E04FF4801383
:109E700012E04FF480630FE04FF480630CE04FF486
:109E8000806309E04FF4806306E0102304E01023B0
:109E900002E0102300E01023D3608CE03C4A7B6892
:109EA0001B6819462D4B994200F083807B681B6824
:109EB00019462B4B99427AD07B681B681946294B6F
:109EC000994272D07B681B681946274B99426AD029
:109ED0007B681B681946254B994261D07B681B68DB
:109EE0001946234B994258D07B681B681946214B71
:109EF00099424FD07B681B6819461F4B994226D068
:109F00007B681B6819461D4B99421DD07B681B68F6
:109F100019461B4B994214D07B681B681946194B94
:109F200099420BD07B681B681946174B994202D1A6
:109F30004FF480133EE04FF080633BE04FF480131A
:109F400038E04FF4801335E04FF4801332E04FF4E3
:109F500080632FE0B860024000640240106002405D
:109F60001064024070600240706402402860024049
:109F700028640240886002408864024040600240D9
:109F800040640240A0600240A06402405860024069
:109F9000006002404FF480630CE04FF4806309E0FE
:109FA0004FF4806306E0102304E0102302E0102346
:109FB00000E0102393607B68312283F835207B68B2
:109FC0001B6C002B03D07B681B6C786898477B6800
:109FD0001B681A46774B9A4272D9774B5A687B684E
:109FE0001B681946754B994262D07B681B681946FD
:109FF000734B99425AD07B681B681946714B994242
:10A0000052D07B681B6819466F4B99424AD07B68D7
:10A010001B6819466D4B994241D07B681B681946F5
:10A020006B4B994238D07B681B681946694B994243
:10A030002FD07B681B681946674B994226D07B68F6
:10A040001B681946654B99421DD07B681B681946F1
:10A05000634B994214D07B681B681946614B994247
:10A060000BD07B681B6819465F4B994202D14FF4B5
:10A0700000131EE04FF000631BE04FF4001318E0E4
:10A080004FF4001315E04FF4001312E04FF4006397
:10A090000FE04FF400630CE04FF4006309E04FF46D
:10A0A000006306E0202304E0202302E0202300E0F8
:10A0B00020231340002B14BF01230023DBB29EE1B9
:10A0C0007B681B681A46494B9A4240F291803A4B92
:10A0D0001A687B681B681946384B994262D07B68C6
:10A0E0001B681946364B99425AD07B681B68194643
:10A0F000344B994252D07B681B681946324B9942C7
:10A100004AD07B681B681946304B994241D07B6826
:10A110001B6819462E4B994238D07B681B6819463C
:10A120002C4B99422FD07B681B6819462A4B9942C9
:10A1300026D07B681B681946284B99421DD07B6846
:10A140001B681946264B994214D07B681B68194638
:10A15000244B99420BD07B681B681946224B9942CD
:10A1600002D14FF400131EE04FF000631BE04FF4E8
:10A17000001318E04FF4001315E04FF4001312E041
:10A180004FF400630FE04FF400630CE04FF4006302
:10A1900009E04FF4006306E0202304E0202302E0FE
:10A1A000202300E020231340002B14BF01230023B1
:10A1B000DBB224E1586402400064024010600240B7
:10A1C00010640240706002407064024028600240E7
:10A1D0002864024088600240886402404060024077
:10A1E00040640240A0600240A0640240B8600240A7
:10A1F0007B681B681A46704B9A4272D96F4B5A683B
:10A200007B681B6819466E4B994262D07B681B685D
:10A2100019466C4B99425AD07B681B6819466A4BA9
:10A22000994252D07B681B681946684B99424AD0C4
:10A230007B681B681946664B994241D07B681B6856
:10A240001946644B994238D07B681B681946624BAB
:10A2500099422FD07B681B681946604B994226D0E3
:10A260007B681B6819465E4B99421DD07B681B6852
:10A2700019465C4B994214D07B681B6819465A4BAF
:10A2800099420BD07B681B681946584B994202D102
:10A290004FF400131EE04FF000631BE04FF4001377
:10A2A00018E04FF4001315E04FF4001312E04FF4E0
:10A2B00000630FE04FF400630CE04FF4006309E02B
:10A2C0004FF4006306E0202304E0202302E0202373
:10A2D00000E020231340002B14BF01230023DBB236
:10A2E0008DE0364B1A687B681B681946344B9942DF
:10A2F0007ED07B681B681946324B99425AD07B68E6
:10A300001B681946304B994252D07B681B6819462E
:10A310002E4B99424AD07B681B6819462C4B9942B8
:10A3200041D07B681B6819462A4B994238D07B681C
:10A330001B681946284B99422FD07B681B68194629
:10A34000264B994226D07B681B681946244B9942BC
:10A350001DD07B681B681946224B994214D07B683C
:10A360001B681946204B99420BD07B681B68194625
:10A370001E4B994202D14FF400133AE04FF00063B4
:10A3800037E04FF4001334E04FF4001331E04FF4A2
:10A3900000132EE04FF400632BE04FF4006328E03D
:10A3A0004FF4006325E04FF4006322E0202320E017
:10A3B00020231EE020231CE0586002400060024081
:10A3C00010600240106402407060024070640240FD
:10A3D000286002402864024088600240886402408D
:10A3E0004060024040640240A0600240A06402401D
:10A3F00020231340002B14BF01230023DBB2002BCA
:10A4000000F045847B681B681B6803F01003002B79
:10A4100000F03D847B681B681B6803F48023002BDD
:10A4200000F00D827B681B681A46A04B9A426CD9DB
:10A430009F4A7B681B6819469E4B994262D07B6895
:10A440001B6819469C4B99425AD07B681B68194679
:10A450009A4B994252D07B681B681946984B994297
:10A460004AD07B681B681946964B994241D07B685D
:10A470001B681946944B994238D07B681B68194673
:10A48000924B99422FD07B681B681946904B99429A
:10A4900026D07B681B6819468E4B99421DD07B687D
:10A4A0001B6819468C4B994214D07B681B6819466F
:10A4B0008A4B99420BD07B681B681946884B99429E
:10A4C00002D14FF400131EE04FF000631BE04FF485
:10A4D000001318E04FF4001315E04FF4001312E0DE
:10A4E0004FF400630FE04FF400630CE04FF400639F
:10A4F00009E04FF4006306E0202304E0202302E09B
:10A50000202300E02023D36076E17B681B681A4695
:10A51000744B9A426CD9664A7B681B681946654B36
:10A52000994262D07B681B681946634B99425AD0A6
:10A530007B681B681946614B994252D07B681B6847
:10A5400019465F4B99424AD07B681B6819465D4BA0
:10A55000994241D07B681B6819465B4B994238D0C1
:10A560007B681B681946594B99422FD07B681B6842
:10A570001946574B994226D07B681B681946554BA4
:10A5800099421DD07B681B681946534B994214D0E1
:10A590007B681B681946514B99420BD07B681B683E
:10A5A00019464F4B994202D14FF400131EE04FF071
:10A5B00000631BE04FF4001318E04FF4001315E0A4
:10A5C0004FF4001312E04FF400630FE04FF4006308
:10A5D0000CE04FF4006309E04FF4006306E0202331
:10A5E00004E0202302E0202300E02023936003E125
:10A5F0007B681B681A463C4B9A4240F291803B4A6A
:10A600007B681B6819462B4B994200F086807B685B
:10A610001B681946284B99427DD07B681B681946F8
:10A62000264B994275D07B681B681946244B99428A
:10A630006DD07B681B681946224B994264D07B68B9
:10A640001B681946204B99425BD07B681B681946F2
:10A650001E4B994252D07B681B6819461C4B99428D
:10A6600049D07B681B6819461A4B994240D07B68D9
:10A670001B681946184B994214D07B681B68194611
:10A68000164B99420BD07B681B681946144B9942B4
:10A6900002D14FF4001341E04FF000633EE04FF46D
:10A6A00000133BE04FF4001338E000BF5864024051
:10A6B000006402401060024010640240706002407A
:10A6C00070640240286002402864024088600240B2
:10A6D000886402404060024040640240A060024042
:10A6E000A0640240B860024058600240006002402E
:10A6F0004FF4001312E04FF400630FE04FF40063D7
:10A700000CE04FF4006309E04FF4006306E02023FF
:10A7100004E0202302E0202300E02023D3606BE04C
:10A72000884A7B681B681946874B994262D07B68D0
:10A730001B681946854B99425AD07B681B6819469D
:10A74000834B994252D07B681B681946814B9942D2
:10A750004AD07B681B6819467F4B994241D07B6881
:10A760001B6819467D4B994238D07B681B68194697
:10A770007B4B99422FD07B681B681946794B9942D5
:10A7800026D07B681B681946774B99421DD07B68A1
:10A790001B681946754B994214D07B681B68194693
:10A7A000734B99420BD07B681B681946714B9942D9
:10A7B00002D14FF400131EE04FF000631BE04FF492
:10A7C000001318E04FF4001315E04FF4001312E0EB
:10A7D0004FF400630FE04FF400630CE04FF40063AC
:10A7E00009E04FF4006306E0202304E0202302E0A8
:10A7F000202300E0202393607B681B681B6803F420
:10A800000023002B09D17B685B6C002B00F03F829A
:10A810007B685B6C7868984739E27B681B681B68CB
:10A8200003F40023002B00F032827B68DB6B002BEB
:10A8300000F02D827B68DB6B7868984727E27B68A5
:10A840001B681B6803F48073002B07D17B681B68AF
:10A850007A681268126822F010021A607B681B681E
:10A860001A46454B9A4240F28B80444A7B681B68EB
:10A870001946354B994262D07B681B681946334BA9
:10A8800099425AD07B681B681946314B994252D085
:10A890007B681B6819462F4B99424AD07B681B681E
:10A8A00019462D4B994241D07B681B6819462B4BAA
:10A8B000994238D07B681B681946294B99422FD0A2
:10A8C0007B681B681946274B994226D07B681B681A
:10A8D0001946254B99421DD07B681B681946234BAE
:10A8E000994214D07B681B681946214B99420BD0C2
:10A8F0007B681B6819461F4B994202D14FF4001325
:10A900001EE04FF000631BE04FF4001318E04FF41B
:10A91000001315E04FF4001312E04FF400630FE052
:10A920004FF400630CE04FF4006309E04FF4006360
:10A9300006E0202304E0202302E0202300E020237F
:10A94000D36090E100600240106002401064024059
:10A950007060024070640240286002402864024037
:10A9600088600240886402404060024040640240C7
:10A97000A0600240A06402405864024000640240AB
:10A980007B681B681A469F4B9A426CD99E4A7B682B
:10A990001B6819469D4B994262D07B681B6819461B
:10A9A0009B4B99425AD07B681B681946994B994238
:10A9B00052D07B681B681946974B99424AD07B68F6
:10A9C0001B681946954B994241D07B681B68194614
:10A9D000934B994238D07B681B681946914B99423A
:10A9E0002FD07B681B6819468F4B994226D07B6815
:10A9F0001B6819468D4B99421DD07B681B68194610
:10AA00008B4B994214D07B681B681946894B99423D
:10AA10000BD07B681B681946874B994202D14FF4D3
:10AA200000131EE04FF000631BE04FF4001318E02A
:10AA30004FF4001315E04FF4001312E04FF40063DD
:10AA40000FE04FF400630CE04FF4006309E04FF4B3
:10AA5000006306E0202304E0202302E0202300E03E
:10AA600020239360FFE07B681B681A46734B9A4271
:10AA70006CD9734A7B681B681946644B994262D053
:10AA80007B681B681946624B99425AD07B681B68E9
:10AA90001946604B994252D07B681B6819465E4B41
:10AAA00099424AD07B681B6819465C4B994241D059
:10AAB0007B681B6819465A4B994238D07B681B68E3
:10AAC0001946584B99422FD07B681B681946564B44
:10AAD000994226D07B681B681946544B99421DD079
:10AAE0007B681B681946524B994214D07B681B68DF
:10AAF0001946504B99420BD07B681B6819464E4B48
:10AB0000994202D14FF400131EE04FF000631BE0A6
:10AB10004FF4001318E04FF4001315E04FF4001346
:10AB200012E04FF400630FE04FF400630CE04FF4C9
:10AB3000006309E04FF4006306E0202304E02023D3
:10AB400002E0202300E02023D3608CE03C4A7B68B5
:10AB50001B6819462D4B994200F083807B681B6867
:10AB600019462B4B99427AD07B681B681946294BB2
:10AB7000994272D07B681B681946274B99426AD06C
:10AB80007B681B681946254B994261D07B681B681E
:10AB90001946234B994258D07B681B681946214BB4
:10ABA00099424FD07B681B6819461F4B994226D0AB
:10ABB0007B681B6819461D4B99421DD07B681B683A
:10ABC00019461B4B994214D07B681B681946194BD8
:10ABD00099420BD07B681B681946174B994202D1EA
:10ABE0004FF400133EE04FF000633BE04FF40013DE
:10ABF00038E04FF4001335E04FF4001332E04FF427
:10AC000000632FE0B8600240006402401060024020
:10AC1000106402407060024070640240286002408C
:10AC2000286402408860024088640240406002401C
:10AC300040640240A0600240A064024058600240AC
:10AC4000006002404FF400630CE04FF4006309E041
:10AC50004FF4006306E0202304E0202302E02023D9
:10AC600000E0202393607B68DA6C7B68DA647B68A1
:10AC7000112283F835207B68002283F834207B681A
:10AC8000DB6B002B03D07B68DB6B78689847083759
:10AC9000BD4680BD80B485B000AFF860B9607A6011
:10ACA0003B60FB681B68FA681268126822F4802215
:10ACB0001A60FB681B683A685A60FB689B68402B07
:10ACC00008D1FB681B687A689A60FB681B68BA68E1
:10ACD000DA6007E0FB681B68BA689A60FB681B686B
:10ACE0007A68DA601437BD465DF8047B704700BFB0
:10ACF00080B485B000AF78607B6803F00703FB6029
:10AD00000C4BDB68BB60BA684FF6FF031340BB60B7
:10AD1000FB681A02BB68134343F0BF6343F400337C
:10AD2000BB60044ABB68D3601437BD465DF8047B42
:10AD3000704700BF00ED00E080B400AF044BDB685B
:10AD400003F4E0631B0A1846BD465DF8047B7047B8
:10AD500000ED00E080B483B000AF0346FB7108490A
:10AD600097F907305B09FA7902F01F02012000FA17
:10AD700002F241F823200C37BD465DF8047B704792
:10AD800000E100E080B483B000AF03463960FB719E
:10AD900097F90730002B0BDA0D49FB7903F00F030D
:10ADA000043B3A68D2B21201D2B20B441A7609E0DF
:10ADB000084997F907303A68D2B21201D2B20B446F
:10ADC00083F800230C37BD465DF8047B704700BF55
:10ADD00000ED00E000E100E080B489B000AFF86071
:10ADE000B9607A60FB6803F00703FB61FB69C3F19C
:10ADF0000703042B28BF0423BB61FB690433062B24
:10AE000002D9FB69033B00E000237B61BB6901229F
:10AE100002FA03F3013B1A46BB681A407B699A4069
:10AE20007B69012101FA03F3013B19467B680B4062
:10AE3000134318462437BD465DF8047B704700BFB6
:10AE400080B483B000AF78607B68013BB3F1807F52
:10AE500001D301230AE0084A7B68013B5360064B9B
:10AE600000229A60044B07221A60002318460C3710
:10AE7000BD465DF8047B704710E000E080B582B00D
:10AE800000AF78607868FFF733FF0837BD4680BDB4
:10AE900080B586B000AF0346B9607A60FB730023CB
:10AEA0007B61FFF749FF78617869B9687A68FFF7D5
:10AEB00093FF024697F90F3018461146FFF762FFDD
:10AEC0001837BD4680BD00BF80B582B000AF0346D5
:10AED000FB7197F907301846FFF73CFF0837BD466E
:10AEE00080BD00BF80B582B000AF78607868FFF7A2
:10AEF000A7FF034618460837BD4680BD80B483B01F
:10AF000000AF78607B68042B06D1094A084B1B68A8
:10AF100043F00403136005E0054A054B1B6823F06A
:10AF2000040313600C37BD465DF8047B704700BF17
:10AF300010E000E080B500AF0E4A0E4B1B6843F4F2
:10AF4000007313600B4A0B4B1B6843F48063136060
:10AF5000084A084B1B6843F4807313600320FFF713
:10AF60008DFF002000F008F8F6F732FD00231846A8
:10AF700080BD00BF003C024080B582B000AF786069
:10AF8000FBF72EFA0246064BA3FB02239B09184649
:10AF9000FFF7A8FF002318460837BD4680BD00BF55
:10AFA000D34D621080B400AF044B1B680133034AD9
:10AFB0001360BD465DF8047B704700BF6001002050
:10AFC00080B400AF034B1B681846BD465DF8047B98
:10AFD000704700BF6001002080B584B000AF78608A
:10AFE0000023FB60FFF7ECFFF86000BFFFF7E8FF0E
:10AFF0000246FB68D21A7B689A42F7D31037BD46E7
:10B0000080BD00BF80B400AF124A124B1B6843F0F2
:10B01000010313600F4B00229A600E4A0D4B1B6810
:10B0200023F0847323F4803313600A4B0A4A5A6076
:10B03000084A084B1B6823F480231360054B002249
:10B04000DA60064B4FF000629A60BD465DF8047B03
:10B05000704700BF003802401030002400ED00E0CF
:10B06000DFF830D0002103E00B4B5B584350043134
:10B070000A480B4B42189A42F6D30A4A02E00023D0
:10B0800042F8043B084B9A42F9D3FFF7BBFFF6F7AF
:10B090004FFB704700C00120E2B200080000002012
:10B0A0004401002044010020980E0020FEE700002B
:10B0B000024B0146186800F04FB800BF4001002065
:10B0C000024B0146186800F003B800BF40010020A1
:10B0D00030B500293CD051F8042C0B1F1D49002A23
:10B0E000B8BF9B180A680C4612B95A600B6030BD95
:10B0F00093420DD219685818904201BF5A585218FD
:10B100001A60426823605A6030BD994203D80A46EB
:10B1100051680029F9D1146815199D420AD11B689C
:10B120002344D0188842136012D108680344136086
:10B130004B680CE002D90C23036030BD1C68181961
:10B14000884201BF08684968001918605960536057
:10B1500030BD00BF6801002070B5CC1C24F0030492
:10B1600008340C2C38BF0C24002C064603DA0C23C0
:10B170003360002070BD8C42F9D3204A136810461A
:10B180001946A1B10A68121B0ED40B2A03D90A6012
:10B190008B188C501FE08B420BBF5A684A680260C4
:10B1A0005A6018BF0B4616E00B464968E9E7144D94
:10B1B0002B681BB9304600F025F828603046214640
:10B1C00000F020F8421C0346D1D0C51C25F0030531
:10B1D00085420AD11C6003F10B001A1D20F0070004
:10B1E000821A0AD05142995070BD3046E91A00F0D7
:10B1F00009F80130BBD02B46ECE770BD6801002098
:10B200006401002038B5064C00230546084623603B
:10B2100000F008F8431C02D1236803B12B6038BD4D
:10B22000940E0020044A05491368002B08BF0B4602
:10B2300018441060184670476C010020980E0020DA
:10B24000008000011F00000053544D2020202020CA
:10B2500050726F64756374202020202020202020ED
:10B26000302E303153544D3332204D61737320539F
:10B27000746F72616765000053544D6963726F6546
:10B280006C656374726F6E696373000030303030C8
:10B290003030303030303141000000004D53432019
:10B2A000436F6E66696700004D534320496E7465B5
:10B2B0007266616365000000000000030080830087
:10B2C0000000000000000000000600000000000078
:10B2D000000000000102030401020304060708093C
:02B2E000430029
:10B2E20089010008AD010008F9010008D101000838
:10B2F200210200084902000871020008120100023E
:10B302000000004083042A570002010203010000EA
:10B3120004030904E53D0008753E0008C13E00082B
:10B3220000000000000000002D4000084D40000811
:10B332000000000000000000000000006D40000856
:10B34200AD400008CD400008ED4000080D41000866
:10B3520009022000010104C0FA09040000020806E3
:10B3620050050705810200020007050102000200E4
:10B3720009022000010104C032090400000208068B
:10B382005005070581024000000705010240000048
:10B3920009072000010104C0320904000002080666
:10B3A2005005070581024000000705010240000028
:10B3B2000A06000200000040010000000024F40020
:10B3C200000000000000000000000000000000007B
:10B3D200000000000000000000000000000000006B
:10B3E200E0B20008000000000000000000000000C1
:10B3F200000000000000000000000000000000004B
:10B40200000000000000000000000000000000003A
:10B41200000000000000000000000000000000002A
:04B42200E000002026
:040000050800B061DE
:00000001FF
